:0200000480007A
:10000000B72F0000938F0F8073900F306F00400365
:100010001300000013000000130000001300000094
:100020001300000013000000130000001300000084
:100030001300000013000000130000001300000074
:100040009702000093824211739052309300000097
:10005000130100009301000013020000930200004E
:100060001303000093030000130400009304000036
:10007000130500009305000013060000930600001E
:100080001307000093070000130800009308000006
:100090001309000093090000130A0000930A0000EE
:1000A000130B0000930B0000130C0000930C0000D6
:1000B000130D0000930D0000130E0000930E0000BE
:1000C000130F0000930F000097110200938101D5D8
:1000D000170502001305056397A503009385458264
:1000E00013060000EF00001A170502001305054C67
:1000F000970502009385455213060000EF00801813
:1001000017B503001305058097B503009385457F58
:1001100037B6ABAB1306B6BAEF00C01617B1030083
:100120001301417EEFB000069392120093D21200A9
:100130009382D2FF638A02008322010013014100EF
:100140006F0000177300203083220100130141006B
:10015000730020301301C1FF23205100F32220340B
:10016000E3C402FC8322010013014100130141F8A2
:1001700023221100232421002326310023284100BB
:10018000232A5100232C6100232E71002320810299
:10019000232291022324A1022326B1022328C10293
:1001A000232AD102232CE102232EF1022320010570
:1001B0002322110523242105232631052328410567
:1001C000232A5105232C6105232E71052320810745
:1001D000232291072324A1072326B1072328C1073F
:1001E000232AD107232CE107232EF107732520347E
:1001F000F3251034130601006F000000731015344E
:1002000083204100032181008321C10003220101D9
:1002100083224101032381018323C10103240102BD
:1002200083244102032581028325C10203260103A1
:1002300083264103032781038327C1030328010485
:1002400083284104032981048329C104032A010569
:10025000832A4105032B8105832BC105032C01064D
:10026000832C4106032D8106832DC106032E010731
:10027000832E4107032F8107832FC1071301C10775
:10028000730020302320C5006376B50013054500B8
:100290006FF05FFF678000000000000000000000BA
:1002A000000000000000000000000000000000004E
:1002B000130101F8232011002322210023243100FF
:1002C0002326410023285100232A6100232C71009A
:1002D000232E8100232091022322A1022324B10294
:1002E0002326C1022328D102232AE102232CF10272
:1002F000232E010323201105232221052324310568
:100300002326410523285105232A6105232C710545
:10031000232E8105232091072322A1072324B1073F
:100320002326C1072328D107232AE107232CF1071D
:100330009702020083A2C22A23A02200F3221034D3
:10034000232E5106EF00C03B170102000321412973
:10035000032101008322C10773901234B7220000E9
:100360009382028873A00230832001000322C1001F
:100370008322010103234101832381010324C1015D
:100380008324010203254102832581020326C10241
:100390008326010303274103832781030328C10325
:1003A000832801040329410483298104032AC10409
:1003B000832A0105032B4105832B8105032CC105ED
:1003C000832C0106032D4106832D8106032EC106D1
:1003D000832E0107032F4107832F81071301010893
:1003E00073002030970202009382C23123A01200D2
:1003F00023A2220023A4320023A6420023A85200F5
:1004000023AA620023AC720023AE820023A09202D2
:1004100023A2A20223A4B20223A6C20223A8D202CC
:1004200023AAE20223ACF20223AE020323A01205A8
:1004300023A2220523A4320523A6420523A85205A0
:1004400023AA620523AC720523AE820523A092077E
:1004500023A2A20723A4B20723A6C20723A8D20778
:1004600023AAE20723ACF207EF6010341701020061
:1004700003210117032101008322C1077390123465
:10048000B72200009382028873A00230832001000B
:100490000322C1008322010103234101832381013F
:1004A0000324C10183240102032541028325810223
:1004B0000326C10283260103032741038327810307
:1004C0000328C103832801040329410483298104EB
:1004D000032AC104832A0105032B4105832B8105CF
:1004E000032CC105832C0106032D4106832D8106B3
:1004F000032EC106832E0107032F4107832F810797
:100500001301010873002030970202009382821FBA
:1005100083A0020003A1420083A1820003A2C200C3
:1005200083A2020103A3420183A3820103A4C201A7
:1005300083A4020203A5420283A5820203A6C2028B
:1005400083A6020303A7420383A7820303A8C2036F
:1005500083A8020403A9420483A9820403AAC20453
:1005600083AA020503AB420583AB820503ACC20537
:1005700083AC020603AD420683AD820603AEC2061B
:1005800083AE020703AFC20983AF82076780000012
:1005900073700430130101F823201100232221007D
:1005A000232431002326410023285100232A6100FF
:1005B000232C7100232E8100232091022322A102EB
:1005C0002324B1022326C1022328D102232AE102D7
:1005D000232CF102232E01032320110523222105C0
:1005E000232431052326410523285105232A6105AB
:1005F000232C7105232E8105232091072322A10797
:100600002324B1072326C1072328D107232AE10782
:10061000232CF1079702020083A282FC23A0220070
:10062000232E1106EF30803417010200032141FB15
:10063000032101008322C10773901234B722000006
:100640009382028873A00230832001000322C1003C
:100650008322010103234101832381010324C1017A
:100660008324010203254102832581020326C1025E
:100670008326010303274103832781030328C10342
:10068000832801040329410483298104032AC10426
:10069000832A0105032B4105832B8105032CC1050A
:1006A000832C0106032D4106832D8106032EC106EE
:1006B000832E0107032F4107832F810713010108B0
:1006C00073002030737004306F00000073104530E9
:1006D000678000007325403073F04330678000006E
:1006E00097070000938747FE232EB5FE2322C5FA05
:1006F000232635F82320F5F8130505F86780000058
:10070000130101FF23261100EF60D006EF20005EE9
:10071000631805008320C1001301010167800000F8
:100720008320C100130101016F304024930785002D
:100730001307F0FF2322F5002324E5002326F5000C
:100740002328F500232005006780000023280500EA
:10075000678000008327450023A2F50003A78700D8
:1007600023A4E50003A787002322B70023A4B70032
:1007700023A8A50083270500938717002320F500F1
:100780006780000003A605009307F0FF13078500AC
:100790006316F6006F008003138707008327470066
:1007A00083A60700E37AD6FE23A2F50023A4B700B0
:1007B00023A4E5002322B70023A8A5008327050072
:1007C000938717002320F5006780000003270501A9
:1007D000832747006FF05FFD0327450083268500D0
:1007E000832705012324D70003278500832645009E
:1007F0002322D70003A747006316A700032785001D
:1008000023A2E7002328050003A507001305F5FF31
:1008100023A0A70067800000032605049387050036
:10082000630406028325C50003274500B385C50080
:100830002326B50063E6E500832505002326B500E1
:10084000138507006F50404F67800000130101FFC0
:100850002324810023261100130405002322910084
:10086000EF30104583278404635AF0048327440241
:1008700063860704930444026F0000028327840404
:100880009387F7FF2324F404832784046358F0023A
:10089000832744026384070213850400EF3040700D
:1008A000E30E05FCEF30101D832784049387F7FFC8
:1008B0002324F40483278404E34CF0FC9307F0FF23
:1008C0002324F404EF301042EF30903E8327440499
:1008D000635AF00483270401638607049304040128
:1008E0006F000002832744049387F7FF2322F40458
:1008F000832744046358F0028327040163840702BA
:1009000013850400EF30C069E30E05FCEF3090164C
:10091000832744049387F7FF2322F40483274404A6
:10092000E34CF0FC9307F0FF2322F404032481003E
:100930008320C10083244100130101016F30903AEC
:10094000630A0508130101FE232C8100130405002E
:10095000232E1100232A910023282101232631016F
:1009600013890500EF30D034832404048325C403A5
:100970008329040013850400EFA080611307F0FFB2
:10098000232C0402B3079540B387F9003385A900EF
:100990002322E4042322A400232434012326F40088
:1009A0002324E404631C09028327040163920704DF
:1009B000EF3050338320C10103248101832441019E
:1009C000032901018329C10013051000130101024D
:1009D00067800000737004306F000000130504018D
:1009E000EFF0DFD413054402EFF05FD46FF05FFC4B
:1009F00013050401EF30C05A93071000E31AF5FA0B
:100A0000EFF01FB96FF0DFFA631605007370043062
:100A10006F000000130101FE232A91002328210109
:100A200023263101232E1100232C8100930405007D
:100A300013890500930906006380050AEFA040555D
:100A400013055505EF50C00E13040500630E05088D
:100A5000930745052320F500232E94022320240527
:100A6000EF301025832404048325C40303290400E4
:100A700013850400EFA0C0519306F0FF232C04025D
:100A8000B30795403307A900B307F9002322D40424
:100A90002322E4002326F4002324D40413050401B4
:100AA00023242401EFF09FC813054402EFF01FC870
:100AB000EF30502323083405130504008320C101BF
:100AC0000324810183244101032901018329C100F9
:100AD000130101026780000013054005EF50400537
:100AE0001304050063160500737004306F000000E6
:100AF000232084006FF05FF66316050073700430E6
:100B00006F0000006376B500737004306F00000062
:100B1000130101FF23248100130620001384050024
:100B20009305000023261100EFF01FEE630C050073
:100B3000232C85028320C1000324810013010101BD
:100B400067800000737004306F000000130101FB28
:100B50002326110423248104232291042320210528
:100B6000232E3103232C4103232A5103232861031D
:100B7000232671032326C10063060528638C0526FE
:100B800093072000639CF6000327C503930710001A
:100B90006306F700737004306F00000013890600CD
:100BA0009384050013040500EF30C070631A05003C
:100BB0008327C10063860700737004306F00000054
:100BC000EF30100F032784038327C403130B0000A7
:100BD000930B20009309F0FF130A0401930A4402C7
:100BE0006364F710630479238327C10063820736A7
:100BF00063160B0013058101EF304055EF30900E66
:100C0000EF20C000EF30D00A8327440463943701FB
:100C100023220404832784046394370123240404D7
:100C2000EF30500C9305C10013058101EF300055E2
:100C300063160530EF30D007032784038327C403EE
:100C40006304F710EF30100AEF3090068327840416
:100C50006346F0026F00000313850A00EF30403452
:100C600063040500EF300061832784049387F7FF56
:100C70002324F404832784046356F000832744026A
:100C8000E39C07FC23243405EF30D005EF305002FD
:100C9000832744046346F0026F00000313050A0033
:100CA000EF30003063040500EF30C05C832744045C
:100CB0009387F7FF2322F404832744046356F0004C
:100CC00083270401E39C07FC23223405EF309001C5
:100CD000EF204027130B1000EF30807D03278403A3
:100CE0008327C403E370F7F00326040463040612A9
:100CF000631A091E0325840093850400EF50C00386
:100D0000832784008326040403274400B387D70085
:100D10002324F40063E4E71083278403832604007C
:100D200003274402938717002324D400232CF402C2
:100D30006300071013054402EF308026930710006C
:100D40006318F50E6F004014EF30C0798325C100A1
:100D500013050A00EF20D077EF30807583278404D5
:100D60006346F0026F00000313850A00EF30402352
:100D700063040500EF300050832784049387F7FF56
:100D80002324F404832784046356F0008327440259
:100D9000E39C07FC23243405EF30C074EF3040712E
:100DA000832744046346F0026F00000313050A0022
:100DB000EF30001F63040500EF30C04B832744046D
:100DC0009387F7FF2322F404832744046356F0003B
:100DD00083270401E39C07FC23223405EF30807055
:100DE000EF204016E31805EEEFF08FFA130B10001A
:100DF0006FF09FEE83270504E38407D873700430F7
:100E00006F000000737004306F00000003260404BC
:100E1000631006088327040063860704832784037E
:100E20000327440293871700232CF402E31407F0EE
:100E3000EF30406B130510008320C10403248104AC
:100E400083244104032901048329C103032A810364
:100E5000832A4103032B0103832BC10213010105E4
:100E60006780000003254400EF3080578327840308
:100E7000032744022322040093871700232CF40243
:100E8000E31A07EAE30605FAEFF08FF06FF05FFA76
:100E90000325C40093850400EF40106A83270404EF
:100EA0000327C40083260400B307F0403307F7008C
:100EB0002326E400637ED70403274400B307F7002A
:100EC0002326F40013072000832744026304E90467
:100ED0000327840313071700232CE402E38A07F493
:100EE0006FF05FE50325C40093850400EF40D064F4
:100EF000832704040327C40083260400B307F040BB
:100F00003307F7002326E400E37ED7FA6FF0DFFA19
:100F10008327440203278403E30C07FA032784038F
:100F20001307F7FF232CE40203278403130717009A
:100F3000232CE402E38E07EE6FF0DFDF13050400DD
:100F4000EFF0DF90EF200000130500006FF0DFEE00
:100F5000EF304059130500006FF01FEE130101FF41
:100F600023229100930405001305400523248100EA
:100F700023261100EF40D03B13040500630C050449
:100F8000232C05029307F0FF2322F504130710001A
:100F900013050501232EE4022324F4042322040074
:100FA0002320040023240400232604002320040417
:100FB00023089404EFF08FF713054402EFF00FF7C6
:100FC00093060000130600009305000013050400BB
:100FD000EFF0DFB7130504008320C1000324810074
:100FE00083244100130101016780000063040504AC
:100FF000130101FF232481002322910023261100E5
:10100000232021010329450013040500EF30802926
:10101000930400006304A9028320C100032481001B
:1010200013850400032901008324410013010101F9
:1010300067800000737004306F0000008327C400D5
:10104000930410009387F7FF2326F400E39607FC30
:10105000930600001306000093050000130504002A
:10106000EFF0DFAE6FF05FFB6302050A63880508EF
:10107000130101FE232C8100232A91002328210142
:1010800023244101232E1100232631019307200040
:101090009384060013090600138A05001304050053
:1010A000639CF6000327C503930710006302F70A49
:1010B000737004306F000000EFF0CFE1032784036A
:1010C0008327C403930905006366F70493040000B3
:1010D00013850900EFF08FDF8320C1010324810114
:1010E0001385040003290101832441018329C100E0
:1010F000032A810013010102678000008327050491
:10110000E38807F6737004306F00000073700430DA
:101110006F00000003260404631E060C83270400EE
:1011200063860712832784031307F0FF9387170052
:10113000232CF402832784046388E70E8327840426
:1011400093041000938717002324F4046FF05FF8D2
:10115000EFF04FD8032784038327C40393090500C6
:101160006360F70603260404E30A06FA0325C400B5
:1011700093050A00EF40503C832704040327C40072
:1011800083260400B307F0403307F7002326E4006A
:101190006378D70003274400B307F7002326F40041
:1011A00093072000E390F4F883278403E38C07F689
:1011B000832784039387F7FF232CF4026FF09FF6B5
:1011C00003260404E30C06F40325C40093050A0077
:1011D000EF409036832704040327C40083260400CD
:1011E000B307F0403307F7002326E400E364D7FA9F
:1011F0006FF09FFBE39C04F60325840093050A002F
:10120000EF4090338327840083260404032744009F
:10121000B387D7002324F400E3E6E7F08327040034
:101220002324F4006FF01FF083274402930410007E
:10123000E38007EA13054402EF209056E30A05E82D
:10124000E30809E8232099006FF09FE80325440094
:10125000EF300019232204006FF0DFEC6302050A6F
:101260008327050463860700737004306F00000055
:1012700083270500638A0708130101FE232C8100E0
:10128000232A91001304050023282101232631017C
:10129000232E110013890500EFF0CFC30327840329
:1012A0008327C40393090500930400006376F702C3
:1012B000832784031307F0FF93871700232CF4027E
:1012C00083278404638AE70483278404930410003B
:1012D000938717002324F40413850900EFF00FBF50
:1012E0008320C10103248101138504000329010126
:1012F000832441018329C10013010102678000009A
:10130000737004306F00000083274500E38607F602
:10131000737004306F000000832744026396070057
:10132000930410006FF05FFB13054402EF20504759
:10133000E30805FEE30609FE930710002320F900E9
:101340006FF01FFE130101FC232E1102232C8102DA
:10135000232A910223282103232631032324410336
:10136000232251032326C10063060528638C05262A
:10137000938A06009389050013040500EF209073FB
:10138000631A05008327C100638607007370043069
:101390006F000000EF30C011832784036394071CA3
:1013A0008327C1006380071013058101EF20105AC5
:1013B0009304F0FF13094402130A0401EF30801272
:1013C000EF10D004EF30C00E8327440463949700DD
:1013D00023220404832784046394970023240404B1
:1013E000EF3040109305C10013058101EF20105923
:1013F00063100524EF30C00B83278403638A070A38
:10140000EF30400EEF30C00A832784046346F002B9
:101410006F00000313050900EF20903863040500F6
:10142000EF205065832784049387F7FF2324F40477
:10143000832784046356F00083274402E39C07FC5F
:1014400023249404EF30000AEF30800683274404FD
:101450006346F0026F00000313050A00EF205034CA
:1014600063040500EF201061832744049387F7FF8E
:101470002322F404832744046356F00083270401E5
:10148000E39C07FC23229404EF30C005EF10902B5F
:10149000EF300002832784036396070C8327C10083
:1014A000E39E07F0EF300004130500006F00800F8B
:1014B000EF30400383270400638807108325C100B1
:1014C00013050900EF20D000EF20907E83278404CD
:1014D0006346F0026F00000313050900EF20502C53
:1014E00063040500EF201059832784049387F7FFD6
:1014F0002324F404832784046356F00083274402E2
:10150000E39C07FC23249404EF20D07DEF20507A45
:10151000832744046346F0026F00000313050A00AA
:10152000EF20102863040500EF20D05483274404E3
:101530009387F7FF2322F404832744046356F000C3
:1015400083270401E39C07FC23229404EF20907975
:10155000EF10501F63040508EF2090758327840364
:10156000E38E07F293850900130504008324C40069
:10157000EFF08FAA63940A088327840303270400EB
:101580009387F7FF232CF40263160700EF20D07C2B
:101590002322A4008327040163920708EF2090749C
:1015A000130510008320C103032481038324410316
:1015B000032901038329C102032A8102832A4102EC
:1015C0001301010467800000EF20906E03254400A2
:1015D000EF201051EF2010716FF05FEEEFE05FFB36
:1015E0006FF09FF783270504E38407D873700430F6
:1015F0006F000000737004306F0000008327440206
:1016000023269400E38C07F813054402EF205019B9
:10161000E30605F8EFE0DFF76FF05FF8130504016C
:10162000EF20101893071000E31AF5F66FF09FFEF5
:1016300013050400EFF08FA1EF10D0101305000088
:101640006FF05FF663000506130101FF232481009C
:101650002320210123261100232291008324450009
:101660001389050013040500EF20D0436380A40410
:1016700093060000130609009305000013050400FB
:10168000EFF05FCC93071000630CF5028320C100DC
:101690000324810083244100032901001301010177
:1016A00067800000737004306F0000008327C4005F
:1016B00013051000938717002326F4006FF01FFD19
:1016C0008327C400938717002326F4006FF01FFCC4
:1016D000630805066386050C130101FE232C8100B7
:1016E000232A9100232821012326310123244101AB
:1016F00013040500232E1100130906009389050029
:10170000EFE05FFD83278403130A050093040000C4
:10171000639C070213050A00EFE05FFB8320C10111
:10172000032481011385040003290101832441015D
:101730008329C100032A8100130101026780000090
:10174000737004306F000000032604046304060273
:101750008325C40083274400B385C5002326B40035
:1017600063E6F500832504002326B40013850900F1
:10177000EF40805C832784031307F0FF9387F7FF14
:10178000232CF402832744046384E7028327440460
:1017900093041000938717002322F4046FF09FF73F
:1017A00083270504E38A07F2737004306F0000009A
:1017B0008327040163960700930410006FF09FF5E0
:1017C00013050401EF20C07DE30805FEE30609FED2
:1017D000930710002320F9006FF01FFE6306050831
:1017E00083270504638A050863840708130101FE43
:1017F000232C8100232A9100232821012324410145
:1018000013040500232E110023263101138A05003D
:10181000EFE05FEC832784031309050093040000C5
:10182000638E07008329C40093050A001305040092
:10183000EFE09FFE930410002326340113050900F6
:10184000EFE0DFE88320C101032481011385040058
:1018500003290101832441018329C100032A810056
:101860001301010267800000737004306F000000F4
:10187000737004306F000000E38C07FE7370043057
:101880006F00000063160500737004306F000000E5
:10189000130101FF232481001304050023261100F6
:1018A000EF20104103248403EF20D0438320C100A4
:1018B0001305040003248100130101016780000067
:1018C00063160500737004306F000000130101FF00
:1018D000232611002324810013040500EF20503D2E
:1018E000832784030324C4033304F440EF20903F90
:1018F000130504008320C1000324810013010101AA
:1019000067800000630605000325850367800000EB
:10191000737004306F0000006308050497870300AC
:10192000938747FA03A747006304E50403A7C700AA
:101930006302E50803A74701630AE50603A7C70199
:101940006302E50603A74702630AE50403A7C7028B
:101950006302E50403A74703630AE50203A7C7037D
:101960006302E5026F40C034737004306F00000002
:101970001307000013173700B387E70023A0070001
:101980006F400033130770006FF0DFFE1307600035
:101990006FF05FFE130750006FF0DFFD130740008C
:1019A0006FF05FFD130730006FF0DFFC13072000BE
:1019B0006FF05FFC130710006FF0DFFB0325C50419
:1019C000678000002326B5046780000003450505F5
:1019D00067800000630805000325850313351500A3
:1019E00067800000737004306F000000630C050016
:1019F000832785030325C5033305F54013351500FB
:101A000067800000737004306F0000009787030048
:101A1000938747EB03A707006300070403A787002A
:101A20006308070403A707016308070403A78701E6
:101A30006308070403A707026308070403A78702D4
:101A40006308070403A70703630C070403A78703BE
:101A500063040704678000001307000013173700B2
:101A6000B387E70023A0B70023A2A7006780000088
:101A7000130710006FF09FFE130720006FF01FFE8A
:101A8000130730006FF09FFD130740006FF01FFD3C
:101A9000130750006FF09FFC130770006FF01FFCDE
:101AA000130760006FF09FFB97870300938787E120
:101AB00003A747006300E50403A7C7006306E50426
:101AC00003A747016306E50403A7C7016306E5040E
:101AD00003A747026306E50403A7C7026306E504FC
:101AE00003A74703630AE50403A7C7036302A70428
:101AF000678000001307000013173700B387E70063
:101B000023A0070067800000130710006FF0DFFEBE
:101B1000130720006FF05FFE130730006FF0DFFD4A
:101B2000130740006FF05FFD130750006FF0DFFCFC
:101B3000130770006FF05FFC130760006FF0DFFBAE
:101B4000130101FF2324810023229100232021017E
:101B500013040500232611009384050013090600D1
:101B6000EF201015032744049307F0FF6314F700D8
:101B700023220404032784049307F0FF6314F7006F
:101B800023240404EF20101683278403639A07009C
:101B9000130609009385040013054402EF20802FEB
:101BA000EF20101183278404635AF0048327440232
:101BB00063860704930444026F00000283278404B1
:101BC0009387F7FF2324F404832784046358F002E7
:101BD000832744026384070213850400EF20403CFE
:101BE000E30E05FCEF200069832784049387F7FF49
:101BF0002324F40483278404E34CF0FC9307F0FFD0
:101C00002324F404EF20100EEF20900A83274404CD
:101C1000635AF004832704016386070493040401D4
:101C20006F000002832744049387F7FF2322F40404
:101C3000832744046358F002832704016384070266
:101C400013850400EF20C035E30E05FCEF20806211
:101C5000832744049387F7FF2322F4048327440453
:101C6000E34CF0FC9307F0FF2322F40403248100EB
:101C70008320C100832441000329010013010101D5
:101C80006F20500697F701009387879583A607007A
:101C900017F70100130787930327070023A2A60065
:101CA000636AE504130101FF232481002326110048
:101CB00017F7010013078792130405000325070097
:101CC00083A5070093854500EFE0DFAB97F70100A0
:101CD0009387078E83A707006376F40097F70100C8
:101CE00023A8878C8320C1000324810013010101F4
:101CF0006780000017F701001307078E0325070010
:101D000083A50700938545006FE0DFA797F70100E3
:101D10009387078D03A7070083A60700832747043F
:101D20009387F7FF2322F70483A7460463940700F1
:101D3000736004306780000063020504130101FD35
:101D4000232E3101232A510123261102938A0700F1
:101D5000232481022322910223202103232C4101E9
:101D6000232861012326710193074000930907008E
:101D700063FAE700737004306F0000007370043082
:101D80006F000000130B0500938405001309060083
:101D9000938B0600130A08006302082C1305000643
:101DA000EF301059130405006302052A13192900A6
:101DB00023284503130609009305500A13050A005A
:101DC000EF40800903C70400832704031309C9FFF8
:101DD000230AE40203C70400338927011379C9FFEA
:101DE0006306070E83C71400A30AF40283C7140016
:101DF000638E070C83C72400230BF40283C72400DF
:101E00006386070C83C73400A30BF40283C7340036
:101E1000638E070A83C74400230CF40283C744007F
:101E20006386070A83C75400A30CF40283C75400D7
:101E3000638E070883C76400230DF40283C7640020
:101E40006386070883C77400A30DF40283C7740078
:101E5000638E070683C78400230EF40283C78400C1
:101E60006386070683C79400A30EF40283C7940019
:101E7000638E070483C7A400230FF40283C7A40062
:101E80006386070483C7B400A30FF40283C7B400BA
:101E9000638E070283C7C4002300F40483C7C40011
:101EA0006386070283C7D400A300F40483C7D40069
:101EB000638E070083C7E4002301F40483C7E400B2
:101EC0006386070083C7F400A301F404130A4400E7
:101ED00013050A00A3010404232634032328340530
:101EE000232A0404EFE09F8613058401EFE01F8698
:101EF00093075000B3873741232C04042328840020
:101F0000232CF4002322840223220404232E04041D
:101F100013860B0093050B0013050900EFE04FFC3F
:101F20002320A40063840A0023A08A007370043075
:101F300017E90100130909698327090097E40100E3
:101F40009384046A638C070003A7040083A704003A
:101F500083274704938717002322F70417E701001C
:101F600013070767832707009387170097E6010089
:101F700023A0F66683A70400638E070E832709005B
:101F8000639C070083A7040083A7C70263E6F900E8
:101F900097E7010023A6876497E70100938787618D
:101FA00083A7070017E70100130707620325C40290
:101FB000032707009387170097E6010023ACF65E1E
:101FC0002324F4046376A70097E7010023AEA75EFD
:101FD00093054001EF80D07B97E701009387477A14
:101FE0003385A70093050A00EFE0CFF683270900A9
:101FF0006388070083A7040083A747046390071240
:102000008327090013041000638A070083A70400D4
:1020100083A7C70263F43701EFE08FD713050400ED
:102020008320C10203248102832441020329010287
:102030008329C101032A8101832A4101032B010164
:10204000832BC100130101036780000013050A0000
:10205000EF3010461304F0FF6FF05FFC13152600FD
:10206000EF30102D130A0500E31A05D21304F0FF18
:102070006FF0DFFA97E7010023A4875603270700D4
:1020800093071000E31AF7F017E501001305456FF9
:10209000EFE0CFE917E501001305C56FEFE00FE9A9
:1020A00017E5010013054570EFE04FE817E5010063
:1020B0001305C570EFE08FE717E5010013054571C3
:1020C000EFE0CFE617EB0100130BCB7113050B000C
:1020D000EFE0CFE597EA0100938A0A7213850A00C0
:1020E000EFE0CFE417E5010013054572EFE00FE4E0
:1020F00017E501001305C572EFE04FE317E5010096
:1021000013054573EFE08FE297E7010023A8674DC1
:1021100097E7010023A2574D6FF01FE803A70400C3
:1021200083A60400832747049387F7FF2322F7043D
:1021300083A74604E39607EC736004306FF05FEC0E
:10214000130101FF23248100232611002322910083
:1021500023202101130405007370043097E401006B
:102160009384444683A70400639E07106318040009
:1021700097E701009387C74603A4070013094400AB
:1021800013050900EFE04FE583278402638607000B
:1021900013058401EFE04FE49305090017E5010002
:1021A00013050568EFE00FDB97E70100938787428F
:1021B00003A7070097E701009387C73F83A707009E
:1021C0001307170097E6010023A6E64003A70400C3
:1021D0009387170097E6010023AEF63C630C0700D7
:1021E00097E701009387C73F03A70700032747042A
:1021F000631C070E83A70400638A070697E70100A4
:102200009387073E03A707006302871073700430AB
:1022100003A704006318070817E701001307073C2A
:102220008326070083A606006392060A1307F0FFC1
:1022300097E6010023AEE63603A704006308070211
:1022400003A70700032747046302070203A7070049
:1022500083A60700832747049387F7FF2322F70409
:1022600083A7460463940700736004308320C10091
:10227000032481008324410003290100130101018B
:102280006780000097E701009387873503A7070061
:1022900083A7070083274704938717002322F704A7
:1022A0006FF0DFEC83A6070003A7070003A746042F
:1022B0001307170023A2E60417E7010013070732EC
:1022C0008326070083A60600E38206F6032707009D
:1022D0000327C7000327C7000327470097E601002D
:1022E00023A8E62C6FF05FF503A7070083A607007D
:1022F000832747049387F7FF2322F70483A7460425
:10230000E39A07EE736004306FF0DFEE97E70100A9
:102310009387C72983A7070063860700737004307B
:102320006F000000032481008320C100832441004A
:1023300003290100130101016FE08FA56304050C5F
:1023400017E701001307C72983260700930700003A
:102350006386A60A130101FF2326110023248100AE
:10236000232291007370043097E60100938686253E
:1023700083A70600638C0700032607008327070056
:1023800083274604938717002322F60483A70600B9
:102390009304050003244501638807008327070091
:1023A00083A747046394070697E7010093870723F1
:1023B00083A70700638C870697E701009387C721EF
:1023C00083A707006384870697E701009387874602
:1023D0006306F40497E7010093878744630CF402D3
:1023E000930710008320C10003248100832441004F
:1023F00013850700130101016780000013850700A2
:1024000067800000737004306F000000EFF01F90D1
:102410006FF09FF9930740006FF0DFFC83A7840201
:1024200093B71700938727006FF0DFFB9307200017
:102430006FF05FFB7370043097E701009387871894
:1024400003A70700631607026304050483A70700B8
:102450000325C502638C070097E70100938747189F
:1024600003A7070003274704631C070267800000D7
:1024700017E701001307C716832607000327070085
:1024800003A746041307170023A2E604E31005FC84
:1024900017E701001307C714032507006FF01FFBA0
:1024A00003A7070083A60700832747049387F7FF46
:1024B0002322F70483A74604E39A07FA73600430E3
:1024C00067800000130101FF23248100130405002D
:1024D00023261100EFE00FA06318040097E7010026
:1024E0009387071003A407000324C402EFE00F9EA4
:1024F0008320C1001305040003248100130101019E
:10250000678000009307400063F6B70073700430E3
:102510006F000000130101FE232C8100232E110007
:10252000232A91002328210123263101232441015C
:10253000130405007370043017E9010013098908BA
:1025400083270900639207106300041283270405A0
:10255000638EF50A17E701001307870863F0B702D7
:1025600083260700638E8612032707008324C70291
:10257000B3B4950093C414006F00000183240700D6
:10258000B384844093B414000327C4026386E70E27
:10259000832784012328B40463C8070093075000ED
:1025A000B385B740232CB40093172700B387E70007
:1025B0000327440197E901009389891C9397270019
:1025C000B387F9006310F704130A440013050A00E7
:1025D000EFE08FA097E70100938707FF0325C40270
:1025E00083A7070063F6A70097E7010023AEA7FCC7
:1025F00093054001EF80D01993050A003385A900A7
:10260000EFE04F9563840400EFD09FF88327090023
:10261000638C070097E70100938787FC83A7070077
:1026200083A74704639E07048320C101032481011B
:1026300083244101032901018329C100032A810068
:10264000130101026780000097E70100938747F9B3
:1026500003A7070083A70700832747049387170072
:102660002322F704E31404EE97E70100938747F76A
:1026700003A407006FF09FED2326B4026FF05FF113
:10268000032481018320C101832441010329010125
:102690008329C100032A8100130101026FF00FE7B3
:1026A000930400006FF05FEE630A0508130101FE5A
:1026B000232A910097E40100938484F283A7040005
:1026C000232E1100232C81002328210123263101F0
:1026D0006388A7047370043017E90100130989EEB9
:1026E00083270900638C070003A7040083A7040065
:1026F00083274704938717002322F7040327450104
:1027000097E7010093870713630EF70283270900F9
:102710006388070083A7040083A74704639E070814
:102720008320C10103248101832441010329010184
:102730008329C10013010102678000007370043017
:102740006F0000008327850217E701001307070CBD
:10275000E38EE7FAE39C07FA9309450013040500AA
:1027600013850900EFE04F8797E701009387C7E5DE
:102770000325C40283A7070063F6A70097E70100BB
:1027800023A4A7E493054001EF80900097E70100A0
:10279000938707FF3385A70093850900EFD09FFB40
:1027A00083A704000327C40283A7C702E360F7F6E8
:1027B000EFD01FDE6FF09FF5032481018320C1015C
:1027C00083244101032901018329C100130101026E
:1027D0006FF0CFD363020506130101FE232C8100A5
:1027E000232A91002326310113040500232E110012
:1027F00023282101EFD01FEE0327440197E70100B2
:10280000938747039309050093040000630AF702C6
:1028100013850900EFD09FEB8320C10103248101C0
:102820001385040003290101832441018329C10088
:102830001301010267800000737004306F00000014
:102840008327840217E50100130545FCE382A7FCFA
:10285000E39007FC97E70100938747D583A707001C
:102860006394070697E70100938787D783A707003C
:102870008324C4021309440083A7C7021305090077
:10288000B3B4F400EFD05FF597E701009387C7D3A7
:102890000325C40283A7070093C4140063F6A700AE
:1028A00097E7010023A2A7D293054001EF80406E75
:1028B00097E701009387C7EC930509003385A700CC
:1028C000EFD05FE96FF0DFF493058401EFD09FE86C
:1028D0006FF01FF4130101FE37150000232E1100C5
:1028E000232C8100232A9100232821012326310152
:1028F0002324410123225101EF3080236306052464
:102900009304050013050006EF3080221304050030
:1029100063000528371600009305500A2328950206
:1029200013850400EF30405383240403B7170000DD
:102930009387C7FFB384F400B7474C459387974408
:1029400093094400232AF40213850900230C04028E
:10295000A30104042326040223280404232A0404D4
:10296000EFD0DFDE13058401EFD05FDE9307500068
:10297000232C040493F4C4FF23288400232CF400A4
:102980002322840223220404232E040413060000BD
:1029900097150000938585EA13850400EFD05FD476
:1029A0002320A4007370043017E90100130989C1C2
:1029B0008327090097E40100938484C2638C070095
:1029C00003A7040083A70400832747049387170005
:1029D0002322F70417E70100130787BF83270700A7
:1029E0009387170097E6010023A4F6BE83A704008F
:1029F0006388070A83270900639C070083A70400F4
:102A000083A7C7026396070097E7010023AA87BC44
:102A100097E70100938707BA83A7070097E60100AD
:102A2000938686BA0327C40283A6060093871700FD
:102A300017E601002320F6B82324F40463F6E60029
:102A400097E7010023A2E7B893172700B387E700B1
:102A50009397270017E50100130585D23305F5008C
:102A600093850900EFD01FCF8327090063880700F3
:102A700083A7040083A74704639A070E83270900EE
:102A80006384070083A70400EF201007930710005A
:102A90006304F512631A050A737004306F000000B6
:102AA00097E7010023AE87B20327070093071000C2
:102AB000E310F7F617E50100130585CCEFD01FC72B
:102AC00017E50100130505CDEFD05FC617E501003E
:102AD000130585CDEFD09FC517E50100130505CE81
:102AE000EFD0DFC417E50100130585CEEFD01FC47A
:102AF00097EA0100938A0ACF13850A00EFD01FC31B
:102B000017EA0100130A4ACF13050A00EFD01FC2CB
:102B100017E50100130585CFEFD05FC117E5010070
:102B2000130505D0EFD09FC017E50100130585D030
:102B3000EFD0DFBF97E7010023A257AB97E7010073
:102B400023AC47A96FF0DFEC8320C101032481018E
:102B500083244101032901018329C100032A810043
:102B6000832A4100130101026780000003A70400CB
:102B700083A60400832747049387F7FF2322F704E3
:102B800083A74604E39C07EE736004306FF01FEFE9
:102B9000032481018320C101032901018329C1008C
:102BA000032A8100832A4100138504008324410104
:102BB000130101026F30C00F737004309307F0FFF0
:102BC00017E701002326F79E0324810197E7010000
:102BD00023AAA79E8320C101832441010329010167
:102BE0008329C100032A8100832A410097E701005D
:102BF00023AE079C130101026FD0CFFE7370043027
:102C000097E7010023A0079C6FD01F9017E70100F2
:102C10001307C79983270700938717002320F7001E
:102C2000678000007370043097E7010093878799ED
:102C300003A707006318070217E7010013070799A6
:102C40000325070083A70700638C070097E70100AF
:102C50009387079903A70700032747046314070214
:102C60006780000017E70100130787978326070096
:102C70000327070003A746041307170023A2E6044F
:102C80006FF09FFB03A7070083A607008327470475
:102C90009387F7FF2322F70483A74604E39207FCF8
:102CA0007360043067800000130101FF23261100C8
:102CB00023248100EFD01FA297E70100938707919B
:102CC00003A40700EFD09FA08320C10013050400D8
:102CD00003248100130101016780000097E70100D0
:102CE0009387078F03A5070067800000130101FD8C
:102CF000232611022324810223229102232021036F
:102D0000232E3101232C4101232A51012328610163
:102D10002326710197E701009387478983A707005E
:102D2000639A070617E701001307478A83270700FE
:102D30009387170097E6010023AAF688832A0700E5
:102D4000638A0A0A97E701009387878683A70700AB
:102D50009304000063FEFA0A97E90100938949A2EF
:102D600017EA0100130ACA8783270A009306100096
:102D700003A7C70293172700B387E700939727009D
:102D8000B389F90083A7090063F4F60293041000E5
:102D90006F00000297E701009387878283A70700EF
:102DA000930400009387170017E70100232AF78098
:102DB00097E701009387878083A707006384070054
:102DC000930410008320C1020324810213850400B0
:102DD00003290102832441028329C101032A8101BD
:102DE000832A4101032B0101832BC100130101033D
:102DF0006780000017D401001304447E8327040079
:102E000083A707006388070C737004306F0000000D
:102E100017D401001304847C97E901009389499633
:102E200017DA0100130ACA7B17DB0100130BCB79F9
:102E30008327040083A70700638007088327040013
:102E400083A7C70003A9C70083274900930B490044
:102E500013850B0063EAFA06EFD01F9883278902D7
:102E60001305890163840700EFD01F978327C902E8
:102E700003270B0093850B00139527003305F500FE
:102E8000131525003385A9006376F70017D70100D5
:102E9000232CF772EFD01F8C83270A000327C90267
:102EA00083A7C702E366F7F88327040093041000A2
:102EB00083A70700E39407F89307F0FF17D70100F3
:102EC0002328F76E6FF05FEA17D701002322F76E11
:102ED0006FF09FE917D701001307077083270400DD
:102EE0000327070097D6010023AAE66E17D7010033
:102EF0002324F76E97D701009387076C83A70700F9
:102F00009387170017D701002328F76A8327040047
:102F100083A70700639A07009307F0FF17D7010004
:102F20002328F7686FF01FE28327040083A7C700F8
:102F300083A7C70083A7470017D70100232AF76696
:102F40006FF05FE097D701009387476603A70700FC
:102F500063160700737004306F000000130101FE58
:102F6000232E1100232C8100232A910023282101E4
:102F70002326310123244101232251012320610111
:102F80007370043097D401009384C46303A70400D2
:102F90006310071203A707001307F7FF97D6010076
:102FA00023A6E66083A70700639E070A97D7010060
:102FB0009387076283A707006386070A97DA0100F1
:102FC000938A0A7C17DA0100130A0A6017D90100F4
:102FD00013090961930910006F00C0013385EA00ED
:102FE000EFD04FF7832709000327C40283A7C70246
:102FF0006374F70683A7CA086380070E83A78A094C
:1030000003A4C70013058401EFD00FFD130B440088
:1030100013050B00EFD04FFC8327C40283260A0060
:1030200093050B00139527003305F50013152500B4
:10303000130705003385AA00E3F2F6FA17D701005B
:103040002324F758EFD00FF1832709000327C40288
:1030500083A7C702E360F7FA97D7010023A0375789
:103060006FF05FF91304000083A70400638C07006E
:1030700097D701009387C75683A7070083A7470404
:1030800063980704130504008320C1010324810110
:1030900083244101032901018329C100032A8100FE
:1030A000832A4100032B0100130101026780000005
:1030B00017D701001307C75283260700032707000D
:1030C00003A746041307170023A2E6046FF09FEC42
:1030D000EFE0DFC36FF01FFB17D401001304444E71
:1030E00083270400638C0702832704001309100060
:1030F00063860702EFF09FBF6306050097D70100C4
:1031000023AE274B832704009387F7FF17D70100CF
:103110002328F74A83270400E39E07FC97D7010082
:103120009387C74903A7070093071000E31CF7F232
:10313000EFD00FC6130410006FF01FF363040502F5
:1031400063960500737004306F00000017D701000C
:103150001307C74583270700638A0700737004308D
:103160006F000000737004306F000000130101FF56
:10317000232481002326110083260700032705004E
:103180009386160017D601002322D64297D6010057
:103190009386C64383A606003304B7002320850028
:1031A00063F0E6046372E40263F0860297D70100DD
:1031B0009387074303A5070013054500EFD0CFE130
:1031C00013050400EFE01FACEFF0DFD7630E05003E
:1031D0008320C100032481001301010167800000E6
:1031E000E366E4FC6FF05FFC032481008320C100F0
:1031F000130101016FD0CFB9630E050017D701008D
:103200001307C73A832707006388070073700430E9
:103210006F0000006FD0CFB7130101FF232611000C
:1032200023248100032707009307050013071700D5
:1032300097D6010023ACE63697D601009386463A2E
:1032400017D70100130787380327070003A50600D7
:103250003304F70013054500EFD00FD81305040021
:10326000EFE05FA2EFF01FCE631A05000324810098
:103270008320C100130101016FD08FB18320C100F1
:10328000032481001301010167800000130101FF85
:10329000232481002326110097D70100938707314B
:1032A00083A70700130400009387170017D70100B6
:1032B000232EF72E97D701009387873183A7070026
:1032C00063ECF50E17DE0100130E0E5197D20100CC
:1032D0009382424A1304000013070000930F10006A
:1032E0001303500A6F00C000130ECEFE6386C21196
:1032F00083278EFF93050700E38807FE8327CEFF11
:1033000083A74700232EFEFE6388C72103AFC700B3
:1033100083A747003307E500930E0000232EFEFE2F
:103320006380C70983A8C700938748032320170138
:103330002322F70083A788042326F7012324F7001C
:1033400083A7C8022328F70083A70805232C0700BA
:10335000232AF70003A8080383470800639A670637
:10336000930708009387170083C60700B3850741BA
:10337000E38A66FE93D525009395050193D5050153
:10338000231EB700938E1E0013070702630C1F0550
:103390008327CEFF83A74700232EFEFEE394C7F9C1
:1033A00083274E00232EFEFE6FF0DFF73304640008
:1033B0006304060023200600EFF0DFB813050400C5
:1033C0008320C100032481001301010167800000F4
:1033D00093050000231EB700938E1E0013070702FB
:1033E000E3181FFB3304D40113175400130ECEFE51
:1033F00093050700E39EC2EF97D701009387071E4E
:1034000003AE070083270E00639E071097D70100C5
:103410009387871C03AE070083270E006392071C67
:1034200017DE0100130ECE3583270E0A6398072698
:1034300083274E0BE38E07F683278E0B97DE010062
:10344000938ECE3F83A7470017D701002326F73E70
:10345000638CD73D83AFC70083A747003307B50010
:103460001303000097D6010023A8F63C130F300089
:10347000930220009308500A6388D70903A5C70068
:10348000930745032320A7002322F7008327850401
:103490002326E7012324F7008327C5022328F7000A
:1034A00083278502638407002326570083270505A9
:1034B000232C0700232AF70003280503834708006D
:1034C000639C1733930708009387170083C6070090
:1034D000B3850741E38A16FF93D52500939505012F
:1034E00093D50501231EB70013031300130707022A
:1034F000E38EAFEA83278E0B83A7470097D60100A0
:1035000023ACF632E39CD7F783270E0C97D6010045
:1035100023A4F6326FF09FF683274E00232EFEFE83
:103520006FF0DFDE83274E00130F8E0083A6470067
:103530002322DE00638CE62DB307E50003A74600D7
:1035400083A2C600930E00002322EE00930F2000FA
:103550001303500A6300EF088328C700138748034A
:1035600023A0170123A2E70003A7880423A6F701DD
:1035700023A4E70003A7C80223A8E70003A70805C0
:1035800023AC070023AAE70003A8080303470800A9
:10359000631A672213070800130717008346070002
:1035A000B3050741E38A66FE93D52500939505018F
:1035B00093D50501239EB700938E1E0093870702C3
:1035C000638C122183264E0003A746002322EE00BF
:1035D000E314EFF80327CE002322EE006FF0DFF7AD
:1035E00083274E00130F8E0083A747002322FE007F
:1035F0006388E72183A2C70083A74700B305B5000E
:10360000930E00002322FE00930F20001303500AA4
:103610006300FF0883A8C7009387480323A0150110
:1036200023A2F50083A7880423A6F50123A4F500AF
:1036300083A7C80223A8F50083A7080523AC0500CB
:1036400023AAF50003A808038347080063946714BE
:10365000930708009387170083C607003387074145
:10366000E38A66FE13572700131707011357070154
:10367000239EE500938E1E00938505026386121338
:1036800083274E0083A747002322FE00E314FFF8A0
:103690008327CE002322FE006FF0DFF783274E0A38
:1036A00017DF0100130F4F1883A7470017D701003A
:1036B000232AF7166382E71783A2C70083A7470070
:1036C000B305B500930E000017D70100232CF714A3
:1036D000930F40001303500A6382E70983A8C700D1
:1036E0009387480323A0150123A2F50083A788042C
:1036F00023A6F50123A4F50083A7C80223A8F5009B
:1037000083A7080523AC050023AAF50003A8080336
:1037100083470800639C670493070800938717009A
:1037200083C6070033870741E38A66FE13572700E5
:103730001317070113570701239EE500938E1E0000
:1037400093850502638E120383274E0A83A74700E1
:1037500017D701002328F70CE392E7F98327CE0A55
:1037600017D701002320F70C6FF05FF71307000055
:10377000239EE500938E1E0093850502E39612FDBD
:1037800083274E0B3304D40193155400E38207C200
:103790006FF09FCA13070000239EE500938E1E0062
:1037A00093850502E39E12ED17DE0100130E4EFD18
:1037B00083270E0A3304D40193155400E38A07C605
:1037C0006FF0DFED93050000239EB700938E1E007F
:1037D00093870702E39812DF97D701009387C7DF2B
:1037E00003AE07003304D4019315540083270E0061
:1037F000E38807C26FF0DFDE930500006FF09FCE15
:103800008327CE002322FE006FF0DFDE8326CE006A
:103810002322DE006FF05FD28327CE0A17D7010084
:103820002322F7006FF05FE983270E0C17D7010002
:103830002324F7006FF01FC2130101FD2322910220
:1038400023202103232E3101232C4101232A51015E
:1038500023286101232671012326110223248102DA
:1038600097D90100938989D417D90100130949F127
:1038700017DA0100130A0AD597DA0100938A4AD6AB
:1038800097DB0100938BCBD497D40100938484D42D
:10389000130B10006F00000283A709000324090A1C
:1038A0009387170017D701002322F7D0EFF08FE995
:1038B000631E040083A70400E39007FE832709002A
:1038C000E37AFBFEEFC0DFCC6FF0DFFE73700430F5
:1038D00083270A00639E07048327C90A03A4C7003D
:1038E00013054400EFC05FEF83A70B009387F7FF3A
:1038F00017D70100232EF7CC83A704009387F7FF87
:1039000017D701002328F7CC83270A006388070014
:1039100083A70A0083A747046398070203250403CB
:10392000EF20003913050400EF2080386FF09FF876
:1039300003A70A0083A70A00832747049387170079
:103940002322F7046FF05FF903A70A0083A60A0099
:10395000832747049387F7FF2322F70483A74604AE
:10396000E39E07FA736004306FF05FFB97D70100A6
:103970009387C7C383A70700639E070E130101FF48
:1039800023261100232481002322910097D70100D0
:1039900023A607C217D70100130787C48327070090
:1039A000B7A6A5A59386565A83A7070383A5070044
:1039B000639ED50003A64700631AB60083A687005E
:1039C0006396C60083A7C700638AD7000325070054
:1039D0008325070093854503EF30007717D7010053
:1039E000130787BE8326070017D40100130444D9A8
:1039F0006F000002832707006386070883270700FC
:103A00009387F7FF97D6010023A0F6BC8326070013
:103A100093972600B387D70093972700B307F40046
:103A200083A70700E38807FC0325070093172500F9
:103A3000B387A700939727003307F4008326470036
:103A400093878700B307F40083A4460023229700DE
:103A5000638EF40283A7C4008320C1000324810085
:103A600017D70100232EF7B683244100130101016B
:103A7000678000009307100017D701002320F7B4D8
:103A800067800000737004306F00000083A444005E
:103A900093054001EF70C04F3305A4002322950029
:103AA0006FF05FFB130101FE23282101232E11007B
:103AB000232C8100232A91002326310113090500BC
:103AC0007370043097D401009384C4AF83A70400BB
:103AD00017D401001304C4B0639C070C63140900DD
:103AE000032904009309490013850900EFC0DFCEC4
:103AF000832789026386070013058901EFC0DFCDA4
:103B00009385090017D501001305C5D2EFC09FC4E6
:103B100083A70400638807008327040083A7470462
:103B20006394070A832704006384270D83A7040096
:103B3000638207067370043083A704006398070E3E
:103B400097D70100938787A903A7070003270700DA
:103B50006310070C9307F0FF17D70100232AF7A47F
:103B600083A70400638807028327040083A7470410
:103B70006382070203270400832604008327470487
:103B80009387F7FF2322F70483A746046394070073
:103B9000736004308320C101032481018324410127
:103BA000032901018329C10013010102678000007C
:103BB0000327040083270400832747049387170003
:103BC0002322F7046FF09FF10327040083260400EB
:103BD000832747049387F7FF2322F70483A746042C
:103BE000E39207F47360043083270400E39027F521
:103BF00083A704006382070697D701009387079B7A
:103C000083A707006388070A737004306F00000001
:103C100083A7070083A7C70083A7C70083A7470020
:103C200017D701002326F7986FF09FF303270400AE
:103C30008327040083274704938717002322F70470
:103C400097D701009387879903A7070003270700E9
:103C5000E30207F06FF0DFFB97D7010093874797E8
:103C600017D701001307C7B183A707000327470B26
:103C70006314F7028320C1010324810197D7010057
:103C800023A0079683244101032901018329C10050
:103C90001301010267800000032481018320C10118
:103CA00083244101032901018329C1001301010279
:103CB0006FF0DFCB032481018320C1018324410104
:103CC000032901018329C100130101026FC05F8C28
:103CD0006306050A130101FF2322910097D4010016
:103CE00093840490232021011389050083A50400F7
:103CF000232611002324810093858501EFC09FA80E
:103D000003A5040013054500EFC01FAD9307F0FFA6
:103D1000630AF90697D701009387478B03A407002E
:103D200003A7040083A7070033042401232287008C
:103D3000636EF40697D701009387478A03A50700AF
:103D400083A5040093854500EFC0DFA397D701004A
:103D50009387078683A707006376F40097D701004F
:103D600023A887848320C100032481008324410089
:103D70000329010013010101678000007370043002
:103D80006F00000083A50400032481008320C1008C
:103D9000832441000329010017D50100130585A9DB
:103DA00093854500130101016FC0DF9A97D7010089
:103DB0009387878203A507000324810083A504005D
:103DC0008320C1008324410003290100938545001D
:103DD000130101016FC01F9B630E050097C701000F
:103DE0009387C77C83A70700639A0700737004302A
:103DF0006F000000737004306F000000130101FFBA
:103E00002322910097C401009384847D03A70400BA
:103E10009387050083A50400B7060080B3E7D700A9
:103E20002326110023248100232CF700938585018C
:103E300013040600EFC01F9203A5040013054500FC
:103E4000EFC09F999307F0FF6304F40297C7010046
:103E50009387C77703A507008320C100832441000F
:103E60003305850003248100130101016FD09FE118
:103E700083A50400032481008320C1008324410022
:103E800017D501001305059B93854500130101011A
:103E90006FC05F8C6308050A130101FF23229100A4
:103EA00097C401009384C473232021011389050062
:103EB00083A5040023261100232481009385850116
:103EC00013040600EFC01F8903A504001305450075
:103ED000EFC09F9093071000630AF40697C7010094
:103EE0009387C76E03A4070003A7040083A70700F6
:103EF0003304240123228700636EF40697C7010070
:103F00009387C76D03A5070083A50400938545002B
:103F1000EFC05F8797C701009387876983A7070072
:103F20006376F40097C7010023A487688320C1004B
:103F300003248100832441000329010013010101AE
:103F400067800000737004306F00000083A50400D8
:103F5000032481008320C100832441000329010040
:103F600017D501001305058D938545001301010147
:103F70006FC04FFE97C701009387076603A5070030
:103F80000324810083A504008320C1008324410011
:103F90000329010093854500130101016FC08FFEC5
:103FA000130101FF23261100232481002322910005
:103FB0008327C50003A4C7006304040A9304840193
:103FC00013850400EFC05F8197C701009387075EE8
:103FD00083A70700639A070893044400138504002D
:103FE000EFC08FFF97C701009387075E0327C402C6
:103FF00083A7070063F6E70097C7010023A6E75CE5
:1040000093172700B387E7009397270017C5010090
:1040100013050577938504003305F500EFC08FF392
:1040200097C701009387C75B83A707000327C402D4
:104030001305000083A7C70263FAE7009307100087
:1040400017C70100232CF756130510008320C10069
:1040500003248100832441001301010167800000D3
:10406000737004306F0000009385040017C50100D1
:104070001305C579EFC00FEE6FF09FFA97C70100E7
:104080009387C75283A707006396070073700430B5
:104090006F000000130101FF23261100232481007B
:1040A00023229100B70700800324C500B3E7F50081
:1040B0002320F50063080408EFC00FF293044400C6
:1040C00013850400EFC04FF197C701009387C74FD6
:1040D0000327C40283A7070063F6E70097C7010020
:1040E00023A4E74E93172700B387E7009397270091
:1040F00017C501001305C5683305F5009385040055
:10410000EFC04FE597C701009387874D83A707004E
:104110000327C4021305000083A7C70263FAE70060
:104120009307100017C70100232AF7481305100052
:104130008320C10003248100832441001301010175
:1041400067800000737004306F0000006304050294
:1041500097C701009387474603A7070097C7010049
:104160009387C74683A707002320E5002322F50095
:1041700067800000737004306F0000006304050E58
:10418000638E050C130101FF2326110023248100F7
:10419000130705007370043097C8010093888842A4
:1041A00083A708006380070297C7010093874743EE
:1041B00083A6070083A7070083A7460493871700F9
:1041C00023A2F60417C301001303434083A705008D
:1041D000032603009306F0FF130400006388D7044E
:1041E00017CE0100130E4E3D03250E0003280700D5
:1041F000832647006306A800130410006378D602E4
:104200003308D640130410006372F80203250E0031
:10421000B387C74003260300B387D70023A0F50068
:104220002320A7002322C7001304000083A708004F
:10423000638C070097C701009387873A83A707001D
:1042400083A7470463940702130504008320C10079
:1042500003248100130101016780000073700430A2
:104260006F000000737004306F000000EFD01FAAD1
:104270006FF09FFD9307100017C701002320F7344C
:1042800067800000630605000325C5046780000001
:104290001305000067800000630405002326B504B1
:1042A0006780000097C701009387873303A5070045
:1042B0006780000097C701009387C73083A7070076
:1042C00013051000638C070097C701009387072E22
:1042D00003A50700133515001315150067800000AE
:1042E000630C0508130101FE232A910097C4010005
:1042F0009384042F83A70400232E1100232C810014
:1043000023282101232631010327C50283A7C702E1
:104310006376F7048327850163CC070083A7040035
:1043200083A6C70293075000B387D740232CF5001C
:1043300093172700B387E7000327450117C901003A
:104340001309094493972700B307F9006308F7029C
:1043500083A7040083A7C7022326F5028320C10197
:104360000324810183244101032901018329C10020
:104370001301010267800000678000009309450077
:104380001304050013850900EFC00FC583A70400BF
:1043900017C70100130747230327070083A7C70296
:1043A0002326F4026376F70017C70100232EF720B7
:1043B000139527003305F50003248101131525000B
:1043C0008320C10183244101938509003305A9009D
:1043D0008329C10003290101130101026FC08FB7B6
:1043E00063060502130101FF232611002324810027
:1043F0002322910097C701009387871E03A407001B
:10440000630AA400737004306F00000013050000FD
:1044100067800000832744056396070073700430AB
:104420006F0000008326C402032704059387F7FF6B
:10443000232AF4046384E600638E0700130500005A
:104440008320C10003248100832441001301010162
:10445000678000009304440013850400EFC0CFB7C9
:104460000325040597C701009387071603A70700D4
:1044700093075000B387A7402326A402232CF400FF
:104480006376A70097C7010023A0A71493054001F6
:10449000EF60103097C701009387872E3385A70000
:1044A00093850400EFC00FAB130510006FF05FF9A8
:1044B0007370043097C701009387C71083A7070064
:1044C0006380070297C701009387871103A707003E
:1044D00083A7070083274704938717002322F70445
:1044E0006780000097C701009387C70D83A7070067
:1044F000638C070297C701009387870E03A7070005
:10450000032747046302070203A7070083A60700E7
:10451000832747049387F7FF2322F70483A74604E2
:1045200063940700736004306780000097C7010040
:104530009387070B03A6070083A6070003A70700BE
:104540009307500083A6C60203258601B387D74090
:10455000232CF7006780000097C701009387470866
:1045600003A70700630A070083A6070003A7460501
:104570001307170023AAE60403A5070067800000BD
:10458000130101FD2320210323261102232481028C
:1045900023229102232E3101130905007370043088
:1045A00097C401009384040283A7040017C4010088
:1045B00013040403639E070A8327040083A7870567
:1045C000639A0700832704001307100023AEE70453
:1045D000639A050E83A704006388070083270400FD
:1045E00083A74704639A07147370043083A70400F9
:1045F000639407068327040003A587056308050065
:10460000630209048327040023AC07048327040002
:1046100023AE070483A704006388070083270400F0
:1046200083A74704639207068320C1020324810203
:1046300083244102032901028329C10113010103DB
:104640006780000003270400832787059387F7FF0F
:10465000232CF7046FF09FFB03270400832704003B
:1046600083274704938717002322F7046FF09FF8EE
:104670000327040083270400832747049387170038
:104680002322F7046FF05FF303270400832604005E
:10469000832747049387F7FF2322F70483A7460461
:1046A000E39407F8736004308320C102032481027D
:1046B00083244102032901028329C101130101035B
:1046C00067800000032504002326B1001305450080
:1046D000EFC08F908325C1009307F0FF6380F5083A
:1046E00097C70100938787EE83A90700032704007B
:1046F00083A70700B389B9002322370163ECF906C9
:1047000097C70100938787ED03A507008325040061
:1047100093854500EFC00F8797C70100938747E94E
:1047200083A7070063F6F90097C7010023A237E9C2
:10473000EFB01FE66FF01FEA032704008326040092
:10474000832747049387F7FF2322F70483A74604B0
:10475000E39C07E8736004306FF01FE983250400D1
:1047600017C501001305050D93854500EFB09FFEA9
:104770006FF01FFC97C70100938707E603A50700AA
:104780008325040093854500EFB0DFFF6FF05FFAEB
:10479000130101FD23202103232E310123261102C1
:1047A0002324810223229102232C41011389050035
:1047B000930906007370043097C40100938484E069
:1047C00083A7040017C40100130484E1639C071449
:1047D00003270400930720000327C7056304F7029B
:1047E000832704001345F5FF03A787053375E5000C
:1047F00023ACA704832704001307100023AEE704AB
:10480000639A060A83A704006388070083270400CD
:1048100083A74704639407167370043083A70400CA
:10482000639E0706638809008327040083A7870522
:1048300023A0F900032704009307100013050000CC
:104840000327C705630EF700832704001349F9FF08
:104850001305100003A787053379E90023AC27056A
:104860008327040023AE070483A70400638807009E
:104870008327040083A747046392070C8320C102A7
:104880000324810283244102032901028329C101F7
:10489000032A81011301010367800000032704003C
:1048A0008327040083274704938717002322F704F4
:1048B0006FF05FF7032504002326D10013054500A0
:1048C000EFB09FF18326C1009307F0FF638AF60CD7
:1048D00097C70100938787CF03AA07000327040027
:1048E00083A70700330ADA00232247016368FA0C22
:1048F00097C70100938787CE03A50700832504008F
:1049000093854500EFB01FE897C70100938747CA1A
:1049100083A707006370FA0A97C7010023AA47C953
:104920006F004009032704008327040083274704FE
:10493000938717002322F7046FF09FE903270400F1
:1049400083260400832747049387F7FF2322F70475
:1049500083A74604E39407F2736004308320C10206
:104960000324810283244102032901028329C10116
:10497000032A81011301010367800000032704005B
:1049800083260400832747049387F7FF2322F70435
:1049900083A74604E39207E8736004306FF0DFE713
:1049A0008325040017C501001305C5E8938545005C
:1049B000EFB05FDAEFB0DFBD6FF0DFE497C7010063
:1049C000938787C103A507008325040093854500CD
:1049D000EFB05FDB6FF01FFE630A050C130101FFF0
:1049E000232611002324810023229100232021016A
:1049F0007370043097C401009384C4BC83A704007F
:104A000063960708638606008327850523A0F600C2
:104A100093070600930620000326C505232ED50420
:104A200013870500130405006382D70A63F4F608B0
:104A3000930530006388B700930540006396B70084
:104A4000630CD610232CE40493071000630CF608C3
:104A50001304100083A70400638C070097C70100AC
:104A6000938707B883A7070083A7470463980706BF
:104A7000130504008320C100032481008324410026
:104A800003290100130101016780000097C701009D
:104A9000938707B503A7070083A707008327470469
:104AA000938717002322F7046FF0DFF5737004304B
:104AB0006F00000093061000E398D7F88327850560
:104AC00033E7B700232CE5046FF01FF88327850533
:104AD00093871700232CF5046FF01FF7EFD00FA377
:104AE0006FF01FF91309440013050900EFB0DFCE82
:104AF00097C70100938747AD0325C40283A707002A
:104B000063F6A70097C7010023A0A7AC9305400157
:104B1000EF60004897C70100938787C63385A700D9
:104B200093050900EFB01FC3832784026386070043
:104B3000737004306F00000097C70100938747AA85
:104B400083A707000327C40283A7C702E3F2E7F0A5
:104B5000EFB01FA46FF0DFEF130400006FF09FEFC2
:104B600063080508130101FE232C8100232A91000C
:104B7000232821012326310123244101232251012D
:104B8000232E110093090700138A060093040600E0
:104B90001389050013040500EFB0DFB3930A050085
:104BA00063060A00832784052320FA000327C4052F
:104BB00093072000232EF4046380F40463FA971013
:104BC000930630006388D400930640006396D400B7
:104BD000630CF70E232C2405930710006312F70AC9
:104BE0008327840263820702737004306F00000021
:104BF000737004306F0000008327840593871700CB
:104C0000232CF4046FF05FFD97C701009387079A88
:104C100083A707006390070A9304440013850400E8
:104C2000EFB09FBB97C701009387079A0325C40283
:104C300083A7070063F6A70097C7010023A6A798DC
:104C400093054001EF60C03497C70100938747B3D5
:104C5000938504003385A700EFB0DFAF97C701004D
:104C60009387079883A707000327C40283A7C70277
:104C700063F8E700638609009307100023A0F9009A
:104C80001304100013850A00EFB05FA4130504009D
:104C90008320C101032481018324410103290101EF
:104CA0008329C100032A8100832A410013010102E4
:104CB000678000009305840117C50100130505B541
:104CC000EFB05FA96FF09FF9130400006FF09FFB36
:104CD00093071000E392F4F08327840533E927015A
:104CE000232C24056FF05FEF630A050E130101FE0C
:104CF000232C8100232A910013040500232631016F
:104D0000232E11002328210193840500EFB09F9CDE
:104D1000930720008326C405232EF40483278405EB
:104D2000130710009309050093871700232CF40440
:104D30006396E60883278402638607007370043055
:104D40006F00000097C701009387478683A707007D
:104D5000639A07081309440013050900EFB0DFA7A1
:104D600097C70100938747860325C40283A70700DE
:104D700063F6A70097C7010023A8A7849305400105
:104D8000EF60002197C701009387879F9305090073
:104D90003385A700EFB01F9C97C701009387478416
:104DA00083A707000327C40283A7C70263F8E700AD
:104DB000638604009307100023A0F40003248101FC
:104DC0008320C101832441010329010113850900C6
:104DD0008329C100130101026FB05F8F737004302B
:104DE0006F0000009305840117C50100130505A29B
:104DF000EFB05F966FF05FFA930705006308050652
:104E00007370043017B701001307C77B83260700B0
:104E1000639E060203A6C705930620001305000043
:104E20006316D60023AE070413051000832707007E
:104E3000638C070097B701009387877A03A7070061
:104E400003274704631C07026780000097B6010030
:104E50009386067903A6060083A6060083264604E9
:104E6000938616002322D6046FF0DFFA97B701006D
:104E70009387077783A707006FF09FF803A70700C2
:104E800083A60700832747049387F7FF2322F704AD
:104E900083A74604E39A07FA736004306780000032
:104EA000130101FB2322910423202105232C41031C
:104EB000232A510323286103232671032326110487
:104EC00023248104232E31032324810323229103ED
:104ED0002320A10317B901001309897117BB010031
:104EE000130B4B7097B401009384047097BA0100C0
:104EF000938ACA6F130A1000930B9000832709004E
:104F000003A707006306071683A7C70083A9070046
:104F1000EFD0DFCFEFD01FD183270B00130C05009C
:104F20006368F50C97B7010023AEA76A130600006B
:104F30006376352303A50400B3858941EFC05FC0C4
:104F4000EFE04F806306051603A5040093060000FA
:104F50001306000093058100EFC0CFBEE30005FA01
:104F600083278100E3C207FE8329010183A749014A
:104F70006386070013854900EFB01F86EFD09FCAF4
:104F800083270B00130C05006362F50C8327810057
:104F900017B7010023288765E3E8FBFAB317FA0087
:104FA00013F707216310072013F7770C6316072AFE
:104FB00093F70702E38A07F813850900EF00504FC3
:104FC0006FF09FF883A7C70003A4C70083AC070056
:104FD0009309440013850900EFB01F808327440222
:104FE00013050400E78007008327C4016386470D8B
:104FF0008327090003A70700E31607FC03A70A009D
:1050000097B6010023A0865F97B6010023A0F65E45
:1050100097B7010023AEE75CEFD0DFF26FF0DFF26D
:1050200083A7C70003A4C70003AD0700930C440087
:1050300013850C00EFB04FFA8327440213050400D8
:10504000E78007008327C401638C470B832709008F
:1050500003A70700E31607FC03A70A0097B60100A1
:1050600023A6F65897B7010023A4E7586FF01FF264
:10507000EFD0DFB9EFD01FBB83270B00130C050067
:10508000E368F5F683A70A0003A50400930900006E
:1050900003A60700B385894117B70100232487556C
:1050A00013361600EFC0DFA9EFD0DFE9E31E05E8F5
:1050B000EFB00FCE6FF05FE983278401938509007D
:1050C000B387FC0063E2FC0883A704006386070241
:1050D000232A0100232C9101232E8100EFF08F9DC4
:1050E00003A5040093060000130600009305410188
:1050F000EFB0DFA5E31E05EE737004306F00000013
:105100008327840193850C00B307FD006362FD08CB
:1051100083A7040063860702232A0100232CA10130
:10512000232E8100EFF00F9903A5040093060000E1
:105130001306000093054101EFB05FA1E31805F0ED
:10514000737004306F000000032509002322F4006F
:1051500023288400EFB00FE36FF09FE9EFD09FDECC
:105160008327090083A7C70003A4C700930C44004A
:1051700013850C00EFB04FE68327C401638A47050F
:105180008327440213050400E78007006FF0DFDB8C
:10519000032509002322F40023288400EFB08FDECA
:1051A0006FF0DFEA8327C10023ACF9006382070AAE
:1051B000B387870123A2F90023A839019385490009
:1051C0006362FC0803A50A00EFB0CFDB6FF0DFD706
:1051D00083278401232884003387F9002322E400F5
:1051E000636AEC04330C3C41636EFC0283A7040049
:1051F00063860702232A0100232C3101232E81001C
:10520000EFF04F8B03A50400930600001306000087
:1052100093054101EFB09F93E31405F673700430DA
:105220006F00000003A50A0093850C00EFB08FD536
:105230006FF01FF50325090093850C00EFB08FD4A4
:105240006FF01FF403250900EFB0CFD36FF0DFCF6D
:10525000737004306F0000008327C10083A68901AA
:1052600023A839013387D70023A2E9006362EC0643
:10527000B307FC4063EAD70683A7490213850900F8
:10528000E780070083A7C901E39047CD83A6890182
:105290008327C10003A70400B387D7006306070272
:1052A000232A0100232CF100232E3101EFF08F80FF
:1052B00003A50400930600001306000093054101B6
:1052C000EFB0DF88E31205C8737004306F00000090
:1052D0006374FC00E372F7FA032509009385490023
:1052E000EFB04FCA6FF05FC603A50A00938549006F
:1052F000EFB04FC96FF05FC5130101FF2324810098
:1053000023261100232291002320210117B401003C
:105310001304842DEFF0CF998327040063840704DE
:10532000EFF04F9C83270400638A07029308000074
:1053300013080000930700001307200093060000E5
:105340001306004097B501009385C50E17050000B0
:10535000130545B5EFC05F9E6314050673700430F6
:105360006F00000017B901001309094E1305090069
:10537000EFB0CFBB97B401009384444E1385040073
:10538000EFB0CFBA130600009305C000130540002C
:1053900097B7010023AE272597B7010023A89724CC
:1053A000EFB08FE617B701002320A724630605029C
:1053B00097B5010093858507EFC04FE56FF05FF665
:1053C0008320C100032481008324410003290100BC
:1053D0001301010167800000737004306F0000004A
:1053E000638A050A130101FD232A5101930A05006E
:1053F0001305C002232481022322910223202103CA
:10540000232E3101232C410123261102232861017F
:10541000232671011309070093890600130A060069
:1054200093840500EF00C07013040500630C0502AF
:10543000EFF00F8897B701009387071B83A707003A
:10544000638E0704EFF00F8A1305440023205401F4
:10545000232C9400232E44012320340323222403ED
:10546000EFB0CFAE130504008320C10203248102F4
:1054700083244102032901028329C101032A8101F6
:10548000832A4101032B0101832BC1001301010376
:1054900067800000737004306F00000097BB01004C
:1054A000938B8B3A13850B00EFB04FA817BB01000D
:1054B000130BCB3A13050B00EFB04FA713060000F8
:1054C0009305C0001305400097B7010023A277138E
:1054D00097B7010023AC6711EFB00FD317B70100E6
:1054E0002324A710630A050097B50100938505F4EE
:1054F000EFC0CFD16FF01FF5737004306F00000064
:10550000630E0506130101FE232C8100232E1100DA
:10551000232A910017B401001304040D832804000A
:1055200013080500130500006380080493040700B6
:105530002322B100138706002324C1002326010182
:105540009306500063C0B604EFE0DFD69307200057
:10555000630EF50403250400930600001306000003
:1055600093054100EFB08FDE8320C1010324810148
:10557000832441011301010267800000737004302D
:105580006F0000009305410093060000130607001A
:1055900013850800EFB05FAD8320C10103248101B2
:1055A00083244101130101026780000003250400E8
:1055B000930600001386040093054100EFB00FD955
:1055C0006FF09FFA63060500032505006780000061
:1055D000737004306F0000006316050073700430B0
:1055E0006F000000130101FF232611002324810016
:1055F00013040500EFE0DFEB032544013334A00082
:10560000EFE05FEE130504008320C1000324810056
:1056100013010101678000006316050073700430F8
:105620006F000000130101FF232481001304050013
:1056300023261100EFE0DFE703240402EFE09FEAF6
:105640008320C1001305040003248100130101011C
:105650006780000063160500737004306F0000005F
:10566000130101FF232481002322910013840500EC
:105670009304050023261100EFE09FE323A084029A
:10568000032481008320C100832441001301010110
:105690006FE05FE5130101FF1305C00123248100C2
:1056A00023261100EF00C04813040500630805001D
:1056B0002320050013054500EFB04F8713050400B4
:1056C0008320C100032481001301010167800000D1
:1056D00063020502B70700FFB3F7F5006386070012
:1056E000737004306F000000639A0500737004301B
:1056F0006F000000737004306F000000130101FEA2
:10570000232C810023282101232631012324410158
:1057100023225101232E1100232A9100930907000F
:1057200013890600930A060013840500130A050076
:10573000EFE05FB8631805006386090073700430FA
:105740006F000000EFD08FCC83240A00B377940061
:10575000631209046382070463880A009347F4FF15
:10576000B3F797002320FA00EFD0CFFD8320C101CB
:1057700003248101138504000329010183244101CD
:105780008329C100032A8100832A410013010102F9
:1057900067800000E302F4FCE38809FCB3355001A4
:1057A0009395850163060900B7070004B3E5F5008A
:1057B00013860900B3E5850013054A00EFE0CFE149
:1057C000EFD04FF863140500EFA09FDCEFE01FD689
:1057D000931765009309050063DA0700B704000119
:1057E0009384F4FFB3F499006FF05FF8EFE05FCCBF
:1057F00083290A00B377340163100902638A070022
:1058000063880A009347F4FFB3F737012320FA00B7
:10581000EFE05FCD6FF09FFCE31CF4FE6FF05FFEE6
:10582000630C0500B70700FFB3F7F500638A0700B4
:10583000737004306F000000737004306F0000005C
:10584000130101FF23248100130405002326110006
:10585000232291002320210113890500EFE05FC579
:10586000832404009345F9FFB3F795002320F40047
:10587000EFE05FC78320C10003248100138504008B
:105880000329010083244100130101016780000006
:10589000130101FF232481001304050023261100B6
:1058A000EFA05FE303240400EFA05FE28320C100C8
:1058B0001305040003248100130101016780000027
:1058C000630C0500370700FFB3F7E500638A0700A4
:1058D000737004306F000000737004306F000000BC
:1058E0006F50407DB70700FFB377F600638607006F
:1058F000737004306F00000063160600737004308C
:105900006F000000130101FE232C810023282101D8
:105910002326310123244101232E1100232A910043
:105920001389060093890500130A05001304060075
:10593000EFE05F98631E050463060900737004308E
:105940006F000000EFD08FAC83240A00938509001C
:1059500013050A00B3E49900EFF09FF6B3779400C3
:10596000630AF40883240A00EFD0CFDD8320C1014D
:1059700003248101138504000329010183244101CB
:105980008329C100032A81001301010267800000FE
:10599000EFD0CFA783240A009385090013050A00DE
:1059A000B3E43401EFF0DFF1B3F7840063848704DC
:1059B000E30A09FAB705000513060900B365B40048
:1059C00013054A00EFE04FC1EFD0CFD763140500B5
:1059D000EFA01FBCEFE09FB593176500930405008F
:1059E00063D40702B70700019387F7FFB3F4F4000D
:1059F0006FF0DFF783270A001344F4FFB3F7870043
:105A00002320FA006FF05FF6EFE09FAA83240A00DC
:105A1000B3779400639887009347F4FFB3F7970038
:105A20002320FA00EFE01FAC6FF0DFFB130101FF52
:105A30002324810023261100130405002322910052
:105A4000EFD0CF9C8327440063860702032504011F
:105A50009304C400631895006F00800303250401BC
:105A600063089502B7050002EFE04FE18327440089
:105A7000E39607FE13050400EF0080230324810052
:105A80008320C10083244100130101016FD08FCB1B
:105A9000737004306F000000630C0500370700FFCF
:105AA000B3F7E500638A0700737004306F000000ED
:105AB000737004306F0000006F50C05F630C05000E
:105AC000B70700FFB3F7F500638A0700737004306F
:105AD0006F000000737004306F000000130101FFBD
:105AE00023248100232291002326110013040500A2
:105AF00093840500EFE0DF9B0327040093C7F4FFC6
:105B0000B377F7002320F400032481008320C10031
:105B100083244100130101016FE0DF9C630605004F
:105B200003258501678000001305000067800000E1
:105B3000130101FF23248100232611001304050013
:105B4000EFD0CF8C97B701009387C7AA83A7070030
:105B5000639C0704B797010017B70100130787D1AB
:105B60009387C7FF97B6010023ACE6A817B70100DB
:105B70002326F7A817B701002320F7D097B7010015
:105B8000938787A717B701002326F7CE9307100046
:105B900017B70100232807A617B70100232E07A473
:105BA00017B701002328F7A463120402EFD08FB9BE
:105BB000EF10C05813040000130504008320C10037
:105BC0000324810013010101678000001305840094
:105BD000937735006398070CB79701001307F5FF1B
:105BE0009387A7FFE3E4E7FC97B60100938646A1FD
:105BF00083A706006F00400103A70700630A0700A0
:105C0000938607009307070003A74700E366A7FEF4
:105C100017B701001307479EE38AE7F803A70700B9
:105C2000130600011384870023A0E60003A74700A2
:105C3000B306A740637ED6023388A7002322D8008C
:105C400023A2A7008325480097B601009386469BB0
:105C50006F0080009306070003A706000326470095
:105C6000E36AB6FE2320E80023A0060103A747004D
:105C700097B70100938787A883A70700B387E740FA
:105C800017B70100232CF7A6EFD0CFABE30204F245
:105C9000130504008320C1000324810013010101C6
:105CA000678000001375C5FF130545006FF0DFF234
:105CB00063080506130101FF232481002326110038
:105CC00013040500EFC09FF4930584FF0326C4FF6F
:105CD00017B701001307C7926F00800013870700F2
:105CE0008327070083A64700E3EAC6FE232CF4FEC1
:105CF0002320B70097B70100938747A003A70700A9
:105D00008327C4FF032481008320C100B387E700F9
:105D100017B701002324F79E130101016FD08FA252
:105D20006780000097B701009387479D03A5070090
:105D300067800000678000003367B5001377370085
:105D400093070500631207049308D6FFB3081501F3
:105D500013070500938605006378150303A8060062
:105D60001307470093864600232E07FFE36817FFBB
:105D70009347F5FFB387170193F7C7FF9387470052
:105D8000B385F500B307F5003306C50063F4C70C0F
:105D90009386450013884700B3B6D70033B8050192
:105DA00033E7F50093C61600134818001377370041
:105DB000B3E60601133717003377D700330EF640EA
:105DC00093861700630807061337AE0063140706AF
:105DD00013532E0013880500938607001307000055
:105DE00083280800130717001308480023A0160192
:105DF00093864600E36667FE1377CEFFB385E50022
:105E0000B387E7006306EE0483C605001387170017
:105E10002380D700637EC70283C61500138727003F
:105E2000A380D7006376C70203C725002381E7005C
:105E300067800000B307F640B387F500938515002F
:105E400003C7F5FF93861600238FE6FEE398F5FE61
:105E50006780000067800000B367C50093F73700D4
:105E6000B308C5006382070E63761511B307A0401F
:105E700093F73700138737009306500093F5F50F1B
:105E8000130815003383A8401306F6FF6374D70088
:105E9000130750006368E60E6380070E2300B50009
:105EA00013071000638EE700A300B500130730004E
:105EB000130825006396E700130835002301B50099
:105EC0001396850033E6C500139705013367E60096
:105ED0003303F34093968501B366D700135623002E
:105EE000B307F5001307000023A0D700130717001E
:105EF00093874700E36AC7FE1377C3FFB307E80041
:105F00006300E3082380B70013871700637C17033F
:105F1000A380B70013872700637617032381B70098
:105F20001387370063701703A381B70013874700F7
:105F3000637A17012382B700138757006374170130
:105F4000A382B7006780000093F5F50F13978500D3
:105F5000B365B700139705013367B700E37415FF06
:105F6000930705009387470023AEE7FEE3EC17FF96
:105F70006780000067800000130805006FF05FF481
:105F800067800000930705006FF0DFF78347050087
:105F900013070500638C07001305150083470500F0
:105FA000E39C07FE3305E540678000001305000011
:105FB00067800000130515008347F5FF93851500E2
:105FC00003C7F5FF63880700E386E7FE3385E740F4
:105FD00067800000930700006FF05FFF93070500E4
:105FE0009385150003C7F5FF93871700A38FE7FE7E
:105FF000E31807FE67800000834605009307000250
:106000006398F6001305150083460500E38CF6FE41
:10601000938756FD93F7D70F638007049307050016
:10602000930500006388060413050000938717009A
:10603000138606FD1317250083C607003305A70046
:10604000131515003305A600E39206FE63840500D0
:106050003305A04067800000938536FD8346150018
:1060600093B5150093071500E39006FC1305000097
:106070006FF0DFFD130500006780000083A70500B7
:106080002380A70083A705009387170023A0F500AE
:106090006780000097A601009386065783A7060035
:1060A000173703001307077E13861700B307F7009F
:1060B0002380A70097A5010023A8C5549307A0003B
:1060C000630AF500930700046308F6001305000057
:1060D00067800000E30C06FE370610F01307170078
:1060E0008347F7FF2320F6F083A706009387F7FF87
:1060F00097A5010023AAF550E39207FE13050000BF
:1061000067800000130101EB232291142320211545
:10611000232A5113232481132326111423248114A9
:10612000232E3113232C41132328611323267113AB
:10613000232291132320A113232EB11193040500D0
:10614000138905002326C100130C5002930A900006
:106150008347090063888703638C070603A4040050
:106160006F008000638607062300F40003A4040088
:10617000130919001304140023A0840083470900A5
:10618000E39287FF034619009308190093860800DD
:10619000130D00029309F0FF130AF0FF130800002B
:1061A000130550059307D6FD93F7F70F13891600D3
:1061B000636EF53A17A701001307C7E4939727000A
:1061C000B387E70083A70700B387E700678007006E
:1061D0008320C1140324811483244114032901144E
:1061E0008329C113032A8113832A4113032B01132B
:1061F000832BC112032C8112832C4112032D011217
:10620000832DC1111301011567800000930C8000DC
:10621000232401009307100063DA071D8327C100C0
:1062200003A40400938B770093F68BFF03AB060067
:1062300083A94600938786002326F10013860C006D
:106240009306000013050B0093850900EF20807270
:106250002328A1009307000063803733930D410189
:10626000930B100013860C009306000013050B001F
:1062700093850900EF2040129306000013860C005E
:10628000130B050093890500EF20C06E8327810062
:1062900023A0AD0093861B00938D4D0063863701CC
:1062A000938B06006FF01FFCE37C9BFF63D24603D9
:1062B000930704002380A70103A40400130AFAFF34
:1062C0009307140023A0F40013840700E3C446FFDF
:1062D00093962B0093070101B386D7006F008002CD
:1062E000938777052300F40003A40400938BFBFF3E
:1062F00093871B001304140023A084009386C6FF19
:10630000E358F0E483A70600E3ECFAFC9387070365
:106310006FF05FFD83A70400930600030327C1000D
:106320002380D70083A7040093064700930C000145
:106330001386170023A0C40013068007A380C7009C
:1063400003A404002324010093070700130414008E
:1063500023A0840003AB0700930900002326D1008B
:106360006FF0DFED8327C10083AC0700938B4700FC
:1063700063880C28635C40259307D002631EFD20D0
:1063800083C70C006388070263D8092483A604002E
:10639000938C1C00130AFAFF2380F60003A4040068
:1063A0001304140023A0840083C70C00E39E07FCA1
:1063B0006352400303A40400930700022300F40087
:1063C00003A40400130AFAFF1304140023A084009A
:1063D000E3160AFE232671016FF09FD723240100E4
:1063E00093071000930CA000E3CA07E38327C100C2
:1063F00003A40400938647006FF0DFF503C6160080
:10640000930609006FF01FDA83A704009306500279
:106410002380D70003A404001304140023A08400E5
:106420006FF01FD3930C0001232401006FF09FDE57
:106430008327C10003C616009306090083A907003D
:10644000938747002326F100E35E0AD4138A0900EC
:106450009309F0FF6FF01FD503C61600130DD0028D
:10646000930609006FF01FD49347FAFF93D7F741C3
:1064700003C61600337AFA00930609006FF09FD224
:1064800003C61600130D0003930609006FF09FD199
:1064900083C51600930906FD93060900938705FD41
:1064A00013860500E3E2FAFA93972900B3893701CE
:1064B0009386160093991900B389B90083C5060025
:1064C000938909FD938705FD13860500E3FEFAFC19
:1064D0006FF09FF70327C10083A7040083260700FE
:1064E000130747002326E1002380D70003A40400FC
:1064F0001304140023A084006FF09FC593071000BD
:1065000063D4070F8327C1009386770093F686FF35
:10651000938786002326F10083A9460083A70600FF
:1065200063DE090E83A604001306D002B307F04011
:106530002380C60003A40400B336F000B309304141
:106540001304140023A08400138B0700B389D940DF
:10655000930CA000232401006FF05FCE03C6160049
:1065600013081800930609006FF0DFC383A7040027
:10657000138908006FF09FE9E3729BCF9307100027
:10658000930B000093061000E3C447D36FF05FD471
:1065900097AC0100938C8CEA9385090013850C005D
:1065A000EF10D007330AAA406352400303A404004B
:1065B0002300A40103A40400130AFAFF1304140027
:1065C00023A08400E3160AFE130A000083C70C0010
:1065D000E38207E0E3CC09DA9389F9FF1307F0FFC0
:1065E000E396E9DA6FF0DFDC8327C100938647008A
:1065F00083A707002326D10093D9F7416FF05FF2FC
:10660000635640019307D002E314FDF897AC0100F4
:10661000938CCCE2930780026FF01FD7138B070097
:10662000930CA0002324010003A404006FF01FC1F9
:10663000130101EB232E3113B70900409387F9FFB3
:106640002324811423229114232C4113232A511330
:1066500023261114232021152328611323267113C7
:1066600023248113232291132320A113232EB1115C
:10667000130A05002324B10017A401001304C4F871
:10668000973A0300938A0A2097A40100938404ADEB
:106690002326F100930550021305A00013080004FF
:1066A000B70610F083470A00638EB7046388070AB1
:1066B00003270400130A1A00130617003387EA00A1
:1066C00097A8010023A2C8F42300F7006380A7085D
:1066D000E31A06FD173703001307C71A130717003D
:1066E0008347F7FF23A0F6F0832704009387F7FF83
:1066F00017A60100232AF6F0E39207FE83470A005B
:10670000E396B7FA83461A0013051A00130705002B
:10671000930B0002130BF0FF130CF0FF13080000A3
:1067200093055005930890009387D6FD93F7F70FD4
:10673000130A170063ECF54493972700B38797007B
:1067400083A70700B3879700678007001737030008
:1067500013074713E31406F86FF0DFF48320C11426
:106760000324811483244114032901148329C113B0
:10677000032A8113832A4113032B0113832BC11294
:10678000032C8112832C4112032D0112832DC11180
:106790001301011567800000930C8000130D0000A9
:1067A0009307100063DA072183278100938777001E
:1067B00093F787FF83AD070003AB4700138787007C
:1067C0002324E10013860C009306000013850D00BE
:1067D00093050B00EF20001A2328A10063086D45E4
:1067E000130941019309100013860C009306000061
:1067F00013850D0093050B00EF10103A13860C0063
:1068000093060000930D0500138B0500EF20801602
:106810002320A9009389190013094900E3166DFD8F
:10682000E3F49DFD13060004B70610F063D489035A
:106830008327040013871700B387FA0097A5010088
:1068400023A4E5DC23807701630AC706130CFCFF51
:10685000E3C089FF8327C1001305C100930890009E
:10686000B386F9009396260093070101B386D700FB
:106870001308A00013030004370610F0E38CA6E011
:1068800083A706009305000363F4F80093057005E1
:1068900003270400B387B700930517003387EA0086
:1068A00017AE01002322BED62300F7006386073708
:1068B000638C65329386C6FF6FF05FFC1737030069
:1068C000130747FC130717008347F7FF23A0F6F0D1
:1068D000832704009387F7FF97A5010023A6F5D22D
:1068E000E39207FE130CFCFF6FF09FF68327040072
:1068F000130600041387170097A5010023A6E5D00F
:10690000B386FA00930500032380B6006308C750DE
:106910009387270097A6010023A8F6CE3387EA00C5
:10692000930680072300D70017370300130787F566
:10693000B70610F06392C702130717008347F7FFEB
:1069400023A0F6F0832704009387F7FF17A6010022
:10695000232CF6CAE39207FE83278100930C0001E3
:10696000130D00009387470003278100130B0000DD
:10697000832D07002324F1006FF0DFE483278100DB
:1069800083AC070013894700638E0C4C6358802B3F
:106990009307D0026394FB3E03C70C0093050700E6
:1069A0006314072A6F00002F93071000930CA000B8
:1069B000130D0000E3CA07DF832781009387470098
:1069C0006FF09FFA832781008346170013070A00A0
:1069D00003AB0700938747002324F100E3560CD450
:1069E000130C0B00130BF0FF6FF01FD4834617003E
:1069F000930BD00213070A006FF01FD39347FCFFDD
:106A000093D7F74183461700337CFC0013070A0035
:106A10006FF09FD183461700930B000313070A0002
:106A20006FF09FD003461700138B06FD13070A0073
:106A3000930706FD93060600E3E2F8FA93172B008E
:106A4000B38767011307170093971700B387C70031
:106A500003460700138B07FD930706FD9306060008
:106A6000E3FEF8FC6FF09FF7832581008327040085
:106A70001306A00003A7050093861700B387FA004A
:106A800017A501002322D5B82380E700138945000C
:106A90006300C736930700046384F62A2324210188
:106AA0006FF05FBF9307100063DE07358327810017
:106AB00013877700137787FF930787002324F1005C
:106AC000032B47008327070063560B3E0327040070
:106AD000130600049306170097A5010023A6D5B25C
:106AE0003387EA009305D0022300B700638CC638D1
:106AF000B307F0403337F000330B6041938D07004C
:106B0000330BEB40930CA000130D00006FF09FCBF4
:106B1000834617001308180013070A006FF0DFC040
:106B20008346170013070A006FF01FC08327040075
:106B3000930600041387170017A601002326E6AC6E
:106B4000B387FA00130650022380C700E314D7B4BA
:106B500017370300130707D3B70610F01307170002
:106B60008347F7FF23A0F6F0832704009387F7FFFE
:106B700017A60100232AF6A8E39207FE6FF09FB143
:106B8000930C0001130D00006FF09FC183270400D8
:106B900093060004130A05001387170017A60100C7
:106BA0002324E6A6B387FA00130650022380C70009
:106BB000E312D7AE173703001307C7CCB70610F0A0
:106BC000130717008347F7FF23A0F6F0832704007D
:106BD0009387F7FF17A601002328F6A2E39207FE8A
:106BE000130A05006FF01FAB17370300130787C99F
:106BF000130717008347F7FF2320F6F083270400CD
:106C00009387F7FF97A5010023A0F5A0E39207FE65
:106C10009386C6FF6FF09FC617370300130787C61A
:106C2000E39805FC9386C6FF6FF05FC5E3FA9DBB52
:106C3000930910006FF01FBF130C000003C70C0076
:106C400093050700E30C07E49308F0FF1305A00089
:106C500013080004B70610F0635E0B0C83270400D2
:106C600013861700B387FA0017A30100232EC398D9
:106C70002380E7006382A5086308060B938C1C0041
:106C800003C70C00130CFCFF93050700E31607FC79
:106C9000E35680E1832704009305000213060004F5
:106CA000B70610F06F00C000130CFCFFE3080CDE09
:106CB00013871700B387FA002380B70017A50100D8
:106CC0002324E59493070700E310C7FE173703005A
:106CD000130747BB130717008347F7FF23A0F6F0FE
:106CE000832704009387F7FF17A50100232EF59053
:106CF000E39207FE6FF05FFB17370300130787B8B7
:106D0000E30E06F6130717008347F7FF23A0F6F0FC
:106D1000832704009387F7FF17A601002326F68E2A
:106D2000E39207FE6FF09FF517370300130787B54F
:106D30006FF05FFD130BFBFFE3121BF36FF05FF5CA
:106D400017370300130707B4B70610F0130717002F
:106D50008347F7FF23A0F6F0832704009387F7FF0C
:106D600017A601002322F68AE39207FE23242101BD
:106D70006FF05F92979C0100938C4C6C93050B0015
:106D800013850C00EF108009330CAC40E35880EB06
:106D90008327040013060004B70610F06F00C0003C
:106DA000130CFCFFE30A0CE813871700B387FA0003
:106DB0002380770197A5010023A8E58493070700A6
:106DC000E310C7FE173703001307C7AB13071700FD
:106DD0008347F7FF23A0F6F0832704009387F7FF8C
:106DE00097A5010023A2F582E39207FE6FF05FFBF7
:106DF00017370300130707A9E39806F4232421019A
:106E00006FF05F89832781001387470083A70700FE
:106E10002324E10013DBF7416FF01FCB173703008A
:106E2000130747A6B70610F0130717008347F7FFAD
:106E300023A0F6F0832704009387F7FF179601003D
:106E40002324F67CE39207FE9307100017970100B6
:106E5000232CF77A93078007173703002304F7A240
:106E60006FF09FAF635680019307D002E394FBF06D
:106E7000979C0100938C8C5C130780029305800221
:106E80006FF09FDC973603009386C69F370610F09D
:106E90009386160003C7F6FF2320E6F003270400BD
:106EA0001307F7FF9795010023A0E576E31207FE8D
:106EB0006FF01FC4938D0700930CA000130D00000A
:106EC0006FF05F90B70710F023A0A7F26F000000EB
:106ED000130101FC130341022322B10293050300B5
:106EE000232E11002324C1022326D1022328E102EC
:106EF000232AF102232C0103232E110323266100F0
:106F0000EFF00FF38320C10113050000130101040A
:106F100067800000130101FB130381032324810216
:106F20002326A100232CC10213040500130603002D
:106F30001305C100232611022322F104232ED102BE
:106F40002320E1042324010523261105232E6100BB
:106F5000EFF04F9B8327C100238007000325C1006A
:106F60008320C102330585400324810213010105FA
:106F700067800000B70710F083A647F403A607F464
:106F800003A747F4E31AD7FEB7160000938606FA64
:106F9000B306D60033B6C600B305E60023A4D7F483
:106FA00023A6B7F467800000B70710F003A747F4E3
:106FB00003A607F483A647F4E31AD7FEB71600002A
:106FC000938606FAB306D60033B6C60023A4D7F4D8
:106FD000B305E60023A6B7F49307000873A0473073
:106FE00067800000130101FF232481002326110084
:106FF000979701009387C7611794010013040461F8
:1070000003A70700832704001306F07C93064706B6
:10701000938747069795010023ACD55E97950100AD
:1070200023A6F55E634AD6008320C10003248100B5
:10703000130101016780000013074789979701003A
:1070400023A8E75CEF009054930710006316F50245
:1070500003270400B71700009387F7761305000095
:10706000E3D4E7FCEFF01FE6032481008320C10096
:10707000130101016FB09FB8179501001305853CFE
:10708000EFF01FE513052000EFF0DFE3032481009C
:107090008320C100130101016FB05FB61795010095
:1070A0001305C53B6FF0DFE2179501001305853B23
:1070B0006FF01FE2130101FF2324810023229100BE
:1070C00023261100B7140000179401001304043A9A
:1070D00093878438130000009387F7FFE39C07FE33
:1070E00013050400EFF0DFDE6FF09FFE13050000D4
:1070F0006F00103C130101FF23261100EF0010491F
:107100001307100093070000631AE5008320C100F5
:107110001385070013010101678000001795010026
:1071200013054532EFF0DFDA8320C100930720001A
:10713000138507001301010167800000737004309C
:107140006F00000067800000737004306F00000063
:10715000979701009387874C03A7070083A74700F1
:10716000130101F92324E1022326F102979701007C
:107170009387474B232861052326710503AB07003E
:1071800083AB4700979701009387474A232C41051B
:10719000232A510503AA070083AA470097970100F5
:1071A0009387474923202107232E310503A9070090
:1071B00083A9470023248105232291052320A105CB
:1071C000232EB103232611062324810623229106B0
:1071D000930D0500930C0000179C0100130C0C4646
:1071E000370D0080232461012326710123284101EA
:1071F000232A5101232C2101232E31010325810053
:107200008325C10003260101832641010324810156
:107210008324C101EF101046130604009386040076
:10722000EF2050662320A1022322B1020325010290
:1072300083254102032681028326C102EF30805359
:107240001306000093060000EF201054634205046B
:107250000325010283254102032681028326C10200
:10726000EF30405103260C0083264C00EF201042E3
:107270003325A000631A0500E3960CF6930710006F
:107280002390FD006FF01FF6930C10006FF09FF538
:107290008327010203284102032681021387070086
:1072A000B3470D018326C10213050700938507002C
:1072B0006FF01FFB130101F997970100938787383F
:1072C0002328610503AB07002326710583AB470024
:1072D0009797010093878737232C410503AA07005E
:1072E00023246101232A510583AA470097970100AF
:1072F00093874736232671012320210703A907001E
:1073000023284101232E310583A94700232A510157
:10731000232C2101232E3101032781008327C10063
:10732000032601018326410123248106232291069D
:10733000032481018324C101232EB1039385070017
:10734000930D05001305070023261106232481054C
:10735000232291052320A105EF20403213060400CB
:1073600093860400EF2010522324A1022326B102A9
:10737000930C0000179C0100130C4C2C370D00805F
:10738000232461012326710123284101232A51016D
:10739000232C2101232E3101032581008325C100E7
:1073A0000326010183264101032481018324C101B5
:1073B000EF20C02C1306040093860400EF20904CAD
:1073C0002320A1022322B1020325010283254102C9
:1073D000032681028326C102EF30C0391306000064
:1073E00093060000EF20503A634205040325010292
:1073F00083254102032681028326C102EF308037B4
:1074000003260C0083264C00EF2050283325A000D3
:10741000631A0500E3960CF6930710002390FD0015
:107420006FF01FF6930C10006FF09FF58327010299
:10743000032841020326810213870700B3470D0189
:107440008326C10213050700938507006FF01FFB19
:10745000130101F72326A102130500052324810847
:107460002322910823202109232E3107232C4107B1
:10747000232A510723286107232671072324810724
:10748000232291072320A107232EB10523261108CB
:10749000EFE00FEA979701009387471C03AB0700C3
:1074A00083AB4700979701009387C71B03AA070088
:1074B00083AA4700979701009387471B03A90700FA
:1074C00083A94700979701009387C71A03A4070071
:1074D00083A44700979701009387471A03A84700A2
:1074E00083A70700130C0500232601012324F100C4
:1074F000979701009387071903A8470083A7070000
:10750000930C0000232A01012328F1009797010022
:107510009387C71703A8470083A70700232E0101FD
:10752000232CF100979701009387C71603A8470003
:1075300083A70700232201032320F102979701006C
:107540009387C71503AD070083AD4700232C0102C5
:10755000232E0102232001042322010423200C00F6
:1075600023220C00032581038325C1031306000099
:1075700093060000EF101010232CA102232EB1025D
:1075800023246C0123267C01032581038325C10369
:1075900013060B0093860B00EF10D00D232CA102D5
:1075A000232EB10223284C01232A5C0103258103E9
:1075B0008325C10313060A0093860A00EF10900B7F
:1075C000232CA102232EB102232C2C01232E3C01BB
:1075D000032581038325C10313060900938609004F
:1075E000EF105009232CA102232EB10223208C027C
:1075F00023229C02032581038325C1031306040073
:1076000093860400EF10100703268100232CA102AB
:107610008326C100232EB1022324CC022326DC02C0
:10762000032581038325C103EF10D0040326010144
:10763000232CA10283264101232EB1022328CC0250
:10764000232ADC02032581038325C103EF10900266
:1076500003268101232CA1028326C101232EB1021E
:10766000232CCC02232EDC02032581038325C103B6
:10767000EF10500003260102232CA10283264102B1
:10768000232EB1022320CC042322DC040325810312
:107690008325C103EF10007E232CA102232EB1020B
:1076A0002324AC052326BC05032581038325C103C0
:1076B00013060D0093860D00EF10C07B232CA10252
:1076C000232EB10203250C0083254C000326010460
:1076D00083264104EF10007A2320A1042322B10461
:1076E00003258C008325CC00032601048326410456
:1076F000EF1040782320A1042322B10403250C01BC
:1077000083254C010326010483264104EF10807673
:107710002320A1042322B10403258C018325CC015D
:107720000326010483264104EF10C0742320A10422
:107730002322B10403250C0283254C0203260104F5
:1077400083264104EF1000732320A1042322B104F7
:1077500003258C028325CC020326010483264104E1
:10776000EF1040712320A1042322B10403250C0350
:1077700083254C030326010483264104EF10806F08
:107780002320A1042322B10403258C038325CC03E9
:107790000326010483264104EF10C06D2320A104B9
:1077A0002322B10403250C0483254C040326010481
:1077B00083264104EF10006C2320A1042322B1048E
:1077C00003258C048325CC0403260104832641046D
:1077D000EF10406A2320A1042322B1040325810372
:1077E0008325C1030326010483264104EF209078FA
:1077F0002324A1042326B104032581048325C10485
:107800001306000093060000EF2000786342050491
:1078100097970100938787E20325810403A6070059
:107820008325C10483A64700EF2040663325A000CE
:10783000631C0500E39C0CD08327C10213071000D2
:107840002390E7006FF09FD0930C10006FF01FD0D3
:1078500097970100938707E50325810403A6070096
:107860008325C10483A64700EF2000721355F5015C
:107870006FF01FFC130101F72326A1021305000579
:10788000232481082322910823202109232E310754
:10789000232C4107232A5107232861072326710738
:1078A00023248107232291072320A107232EB1053A
:1078B00023261108EFE0CFA797970100938707DFF2
:1078C00003AB070083AB470097970100938787DEE0
:1078D00003AA070083AA470097970100938707DE52
:1078E00003A9070083A9470097970100938787DDC5
:1078F00003A4070083A4470097970100938707DD3F
:1079000003A8470083A70700130C050023220101E9
:107910002320F100979701009387C7DB03A8470056
:1079200083A70700930C0000232601012324F10004
:1079300097970100938787DA03A8470083A707007A
:10794000232A01012328F10097970100938787D903
:1079500003A8470083A70700232E0101232CF10071
:1079600097970100938787D803A8470083A707004C
:10797000232201032320F10297970100938787D7E1
:1079800003AD070083AD4700232C0102232E010223
:10799000232001042322010423206C0123227C01E3
:1079A000032581038325C10313060B0093860B0077
:1079B000EF10404C232CA102232EB10223244C01B2
:1079C00023265C01032581038325C10313060A00D6
:1079D00093860A00EF10004A232CA102232EB10245
:1079E00023282C01232A3C01032581038325C1037D
:1079F0001306090093860900EF10C047232CA1024B
:107A0000232EB102232C8C00232E9C0003258103FE
:107A10008325C1031306040093860400EF108045FC
:107A200003260100232CA10283264100232EB1024C
:107A30002320CC022322DC02032581038325C103FA
:107A4000EF10404303268100232CA1028326C100AE
:107A5000232EB1022324CC022326DC02032581033A
:107A60008325C103EF10004103260101232CA1024D
:107A700083264101232EB1022328CC02232ADC02D3
:107A8000032581038325C103EF10C03E0326810136
:107A9000232CA1028326C101232EB102232CCC0268
:107AA000232EDC02032581038325C103EF10803CD4
:107AB00003260102232CA10283264102232EB102B8
:107AC0002320CC042322DC04032581038325C10366
:107AD000EF10403A232CA102232EB1022324AC053F
:107AE0002326BC05032581038325C10313060D004E
:107AF00093860D00EF100038232CA102232EB10233
:107B000003250C0083254C00032601048326410431
:107B1000EF1040362320A1042322B10403258C005A
:107B20008325CC000326010483264104EF10803412
:107B30002320A1042322B10403250C0183254C0139
:107B40000326010483264104EF10C0322320A10440
:107B50002322B10403258C018325CC0103260104D3
:107B600083264104EF1000312320A1042322B10415
:107B700003250C0283254C020326010483264104BD
:107B8000EF10402F2320A1042322B10403258C02EF
:107B90008325CC020326010483264104EF10802DA7
:107BA0002320A1042322B10403250C0383254C03C5
:107BB0000326010483264104EF10C02B2320A104D7
:107BC0002322B10403258C038325CC03032601045F
:107BD00083264104EF10002A2320A1042322B104AC
:107BE00003250C0483254C04032601048326410449
:107BF000EF1040282320A1042322B10403258C0484
:107C00008325CC040326010483264104EF1080263B
:107C10002320A1042322B104032581038325C1036A
:107C20000326010483264104EF20D0342324A10439
:107C30002326B104032581048325C1041306000013
:107C400093060000EF20403463420504979701003B
:107C50009387C79E0325810403A607008325C104DB
:107C600083A64700EF2080223325A000631C050077
:107C7000E39C0CD08327C102130710002390E70078
:107C80006FF09FD0930C10006FF01FD097970100FA
:107C9000938747A10325810403A607008325C10418
:107CA00083A64700EF20402E1355F5016FF01FFC0F
:107CB000130101FF232481001307050013040500AD
:107CC0009308000013080000930700009796010036
:107CD0009386469413060040978501009385457A64
:107CE00017F5FFFF1305054723261100EFA0CF84EA
:107CF0001307040093080000130800009307000016
:107D000097960100938626911306004097850100FF
:107D10009385857717F5FFFF1305055AEFA0CF81EF
:107D200013070400930800001308000093070000E5
:107D3000979601009386468E1306004097850100B2
:107D40009385057517050000130505B3EF90DFFE59
:107D500013070400032481008320C100930800005E
:107D60001308000093070000979601009386E68AA7
:107D700013060040978501009385057217F5FFFFF4
:107D80001305456D130101016F901FFB97960100CC
:107D900083D646881307100097970100938787873B
:107DA000130500006398E600179701002314078667
:107DB0001305100003D72700930610006386E60220
:107DC00003D7470093061000130500006388E602FE
:107DD00083D767001307100013050000630AF7023A
:107DE0001305000067800000179701002315078224
:107DF00003D7470093061000E39CE6FC17970100A9
:107E0000231C078083D7670013071000E31AF7FCD1
:107E1000979701002393078067800000B305B500A2
:107E2000930705006386B70003C7070063160700C2
:107E30003385A74067800000938717006FF09FFE8F
:107E4000130101FB23229104232C410323229103DC
:107E5000232611042324810423202105232E31030A
:107E6000232A51032328610323267103232481033A
:107E70002320A103232EB101930C0500138A0500D2
:107E80009304000063DE05003305A0403337A000F3
:107E9000B305B040930C0500338AE5409304F0FF2E
:107EA00063DA06003306C040B337C000B306D040E3
:107EB000B386F640930A06009389060013840C00EB
:107EC00013090A0063960628178B0100130B0B4653
:107ED0006370CA16B70701006372F6149307F00FB8
:107EE00063F4C70093098000B3573601330BFB00DE
:107EF00083470B0013050002B3873701B309F54030
:107F0000638C0900B3153A01B3D7FC00B31A3601EC
:107F100033E9B70033943C0113DB0A0193050B00EE
:107F200013050900EF30000E130A050093050B003E
:107F3000939B0A0113050900EF30400893DB0B0106
:107F40009305050013850B00EF308004131A0A0116
:107F500093570401B367FA0063FAA700B387570188
:107F600063E6570163F4A700B38757013389A7403D
:107F700093050B0013050900EF30C008130A050034
:107F800093050B0013050900EF304003131404019F
:107F900093050500131A0A0113850B0013540401FD
:107FA000EF20107F33648A00637AA4003304540105
:107FB000636654016374A400330454013304A44081
:107FC0003354340193050000638A04003304804075
:107FD000B3378000B305B040B385F5401305040006
:107FE0008320C10403248104832441040329010460
:107FF0008329C103032A8103832A4103032B01033D
:10800000832BC102032C8102832C4102032D010228
:10801000832DC1011301010567800000B70700012E
:1080200093090001E362F6EC930980016FF0DFEB46
:10803000631A06009305000013051000EF20107866
:10804000930A0500B707010063FAFA0E9307F00FD1
:1080500063F4570193098000B3D73A01330BFB0057
:1080600083470B001305000233095A41B3873701D8
:10807000B309F540E38209EAB39A3A01335BFA00A7
:10808000B3153A01B3D7FC0093DB0A0133E9B7001B
:1080900013050B0093850B00EF20D076130A050023
:1080A00093850B00139C0A0113050B00EF20107140
:1080B000135C0C019305050013050C00EF20506DB7
:1080C000131A0A0193570901B367FA0033943C016C
:1080D00063FAA700B387570163E6570163F4A7006B
:1080E000B3875701338BA74093850B0013050B0013
:1080F000EF205071130A050093850B0013050B0048
:10810000EF20D06B9305050013050C00EF2050689D
:1081100093160901131A0A0193D60601B366DA0011
:1081200063FAA600B386560163E6560163F4A6001F
:10813000B38656013389A6406FF01FDEB7070001F2
:1081400093090001E3EAFAF0930980016FF0DFF090
:108150006376DA0093050A006FF01FE7B7070100A6
:1081600063FAF604930BF00F33B5DB0013153500FB
:1081700033D7A600978701009387471BB387E70093
:1081800083CB070093050002B38BAB00338B7541A3
:10819000631C0B0263E4460163EACC003384CC40E9
:1081A000B306DA4033B98C003389264193050900C0
:1081B0006FF09FE1B707000113050001E3EAF6FA4B
:1081C000130580016FF0DFFAB3966601335D760127
:1081D000336DDD00B35D7A01B3156A0133DC7C01D8
:1081E00013540D01336CBC0013850D00930504007E
:1081F000B3196601EF201061930A0500930504008E
:1082000013850D0033996C01931C0D01EF20105B59
:1082100093DC0C01130A05009305050013850C007F
:10822000EF201057939A0A0113570C0133E7EA0025
:10823000930D0A00637EA7003307A701930DFAFF91
:108240006368A7016376A700930DEAFF3307A701D0
:10825000330AA7409305040013050A00EF20905A43
:1082600093050400930A050013050A00EF2010553A
:10827000930505001304050013850C00EF205051F1
:1082800093150C01939A0A0193D50501B3E5BA0041
:108290001307040063FEA500B385A5011307F4FFCF
:1082A00063E8A50163F6A5001307E4FFB385A50104
:1082B000939D0D01B70C0100B3EDED001384FCFF9D
:1082C000B3F78D0033F48900338AA5401385070086
:1082D000930504002326F10093DD0D01EF20504BA0
:1082E00093050400930A050013850D00EF20504A02
:1082F00013DC090193050C002324A10013850D0054
:10830000EF2010498327C10013040C0093050400DB
:10831000130C050013850700EF209047832681008A
:1083200013D70A013305D5003307A7006374D700BC
:10833000330C9C01B70701009387F7FF93550701A2
:108340003377F70013170701B3F7FA00B3858501F8
:10835000B307F7006366BA00631EBA00637CF900D6
:1083600033863741B3B7C700B385A541B385F54020
:1083700093070600B307F9403339F900B305BA4053
:10838000B385254133947501B3D767013364F40095
:10839000B3D565016FF05FC3130101FD2322910284
:1083A000232A5101232611022324810223202103A1
:1083B000232E3101232C4101232861012326710141
:1083C00023248101232291012320A101930A050086
:1083D00093840500639E0638130406009309050084
:1083E00017890100130989F463F8C512B707010062
:1083F000138B05006378F6101307F00F3337C700AF
:1084000013173700B357E6003309F9008346090014
:108410003387E60093060002B386E640638C0600CD
:10842000B394D40033D7EA003314D600336B9700EB
:10843000B399DA00935A040193850A0013050B00DF
:10844000EF20503C1309050093850A00931B04019B
:1084500013050B00EF20903693DB0B01930405000E
:108460009305050013850B00EF20903213190901C5
:1084700093D70901B367F900138A040063FEA700CC
:10848000B3878700138AF4FF63E8870063F6A700C9
:10849000138AE4FFB3878700B384A74093850A005B
:1084A00013850400EF2010361309050093850A0098
:1084B00013850400EF20903093990901930405007F
:1084C000930505001319090113850B0093D90901C0
:1084D000EF20102CB36939011386040063FCA90056
:1084E000B30934011386F4FF63E6890063F4A9003D
:1084F0001386E4FF13140A013364C400130A000056
:108500006F000013B707000113070001E36CF6EEDC
:10851000130780016FF01FEF138A0600631A06002D
:108520009305000013051000EF20502913040500E7
:10853000B7070100637EF4129307F00F63F487001E
:10854000130A8000B35744013309F90003470900B7
:108550009306000233074701B386E6406394061290
:10856000B3848440130A1000135B040193050B00CD
:1085700013850400EF2010291309050093050B0053
:1085800013850400931B0401EF20502393DB0B01A0
:10859000930405009305050013850B00EF20501F81
:1085A0001319090193D70901B367F900938A0400ED
:1085B00063FEA700B3878700938AF4FF63E8870010
:1085C00063F6A700938AE4FFB3878700B384A740CC
:1085D00093050B0013850400EF20D022130905003A
:1085E00093050B0013850400EF20501D939909019A
:1085F00093040500930505001319090113850B0069
:1086000093D90901EF20D018B3693901138604000A
:1086100063FCA900B30934011386F4FF63E6890003
:1086200063F4A9001386E4FF13940A013364C400C1
:108630001305040093050A008320C102032481026C
:1086400083244102032901028329C101032A8101F4
:10865000832A4101032B0101832BC100032C8100DC
:10866000832C4100032D01001301010367800000EA
:10867000B7070001130A0001E366F4EC130A800156
:108680006FF05FEC3314D40033DAE400B399DA000E
:1086900033D7EA00935A0401B394D40093850A00B7
:1086A00013050A00336B9700EF20D015130905005E
:1086B00093850A0013050A00931B0401EF20101094
:1086C00093DB0B01930405009305050013850B0054
:1086D000EF20100C1319090113570B013367E90040
:1086E000138A0400637EA70033078700138AF4FF10
:1086F000636887006376A700138AE4FF3307870067
:10870000B304A74093850A0013850400EF20900F5F
:108710001309050093850A0013850400EF20100A51
:10872000930405009305050013850B00EF20500608
:1087300013170B011357070113190901B367E90058
:108740001387040063FEA700B38787001387F4FF35
:1087500063E8870063F6A7001387E4FFB387870009
:10876000131A0A01B384A740336AEA006FF0DFDF0F
:1087700063ECD51EB707010063F4F6041307F00F8E
:10878000B335D7009395350033D7B60097870100EE
:108790009387C7B9B387E70003C70700130A00022E
:1087A0003307B700330AEA4063160A0213041000C5
:1087B000E3E096E833B6CA00134416006FF05FE7B3
:1087C000B707000193050001E3E0F6FC9305800183
:1087D0006FF09FFBB35CE600B3964601B3ECDC00A0
:1087E00033D4E40093DB0C01B397440133D7EA00A0
:1087F00093850B0013050400336BF700B319460192
:10880000EF2050001309050093850B0013050400A9
:10881000139C0C01EF20807A135C0C01930405007B
:108820009305050013050C00EF208076131909014C
:1088300013570B013367E90013840400637EA7001C
:10884000330797011384F4FF636897016376A700E9
:108850001384E4FF33079701B304A74093850B000B
:1088600013850400EF20007A1309050093850B009F
:1088700013850400EF208074930405009305050020
:1088800013050C00EF20C07093170B011319090199
:1088900093D70701B367F9001386040063FEA700AE
:1088A000B38797011386F4FF63E8970163F6A70087
:1088B0001386E4FFB387970113140401B70B01007B
:1088C0003364C4001389FBFF337D240133F929018C
:1088D000B384A7409305090013050D00EF20406BFA
:1088E000935C040193050900130B050013850C002C
:1088F000EF20006A93D90901130C05009385090044
:1089000013850C00EF20C06813090500938509004A
:1089100013050D00EF20C0673305850193570B0148
:108920003385A700637485013309790193570501E5
:10893000B387270163E6F402E392F4BCB7070100B2
:108940009387F7FF3375F50013150501337BFB00A3
:1089500033964A0133056501130A0000E37AA6CC79
:108960001304F4FF6FF09FB9130A00001304000012
:108970006FF01FCC130101FB2324810423229104F7
:10898000232E3103232291032326110423202105C2
:10899000232C4103232A5103232861032326710337
:1089A000232481032320A103232EB101930C05006E
:1089B000938905001304050093840500639E062631
:1089C00013090600138A0600978A0100938A0A9603
:1089D00063F4C514B70701006376F6129307F00F2E
:1089E00063F4C700130A8000B3574601B38AFA0044
:1089F00003C70A001305000233074701330AE540A5
:108A0000630C0A00B395490133D7EC0033194601D2
:108A1000B364B70033944C01935A090193850A005B
:108A200013850400EF20005E9309050093850A007A
:108A3000131B090113850400EF204058135B0B0141
:108A40009305050013050B00EF208054939909014D
:108A500093570401B3E7F90063FAA700B38727012E
:108A600063E6270163F4A700B3872701B384A74017
:108A700093850A0013850400EF20C0589309050070
:108A800093850A0013850400EF204053131404015A
:108A9000930505009399090113050B001354040174
:108AA000EF20004F33E48900637AA40033042401EB
:108AB000636624016374A400330424013304A440D6
:108AC00033554401930500008320C104032481042D
:108AD00083244104032901048329C103032A810358
:108AE000832A4103032B0103832BC102032C810240
:108AF000832C4102032D0102832DC10113010105C5
:108B000067800000B7070001130A0001E36EF6EC6E
:108B1000130A80016FF05FED631A060093050000F1
:108B200013051000EF20804913090500B707010065
:108B3000637AF90E9307F00F63F42701130A80009C
:108B4000B3574901B38AFA0003C70A0013050002AC
:108B5000B384294133074701330AE540E30E0AEAAB
:108B600033194901B3DAE900B395490133D7EC0071
:108B700093540901336BB70013850A0093850400F1
:108B8000EF2040489309050093850400931B0901D9
:108B900013850A00EF20804293DB0B01930505004B
:108BA00013850B00EF20C03E9399090193570B01E9
:108BB000B3E7F90033944C0163FAA700B3872701A8
:108BC00063E6270163F4A700B3872701B38AA740B0
:108BD0009385040013850A00EF20C0429309050025
:108BE0009385040013850A00EF20403D930505009E
:108BF00013850B00EF20C03993150B0193990901E0
:108C000093D50501B3E5B90063FAA500B385250145
:108C100063E6250163F4A500B3852501B384A5406F
:108C20006FF09FDFB7070001130A0001E36AF9F054
:108C3000130A80016FF0DFF0E3E8D5E8B707010021
:108C400063FCF604930BF00F33B5DB00131535000E
:108C500033D7A600977701009387476DB387E70066
:108C600083CB070093050002B38BAB00338B7541B8
:108C7000631E0B0263E4360163EACC003384CC400C
:108C8000B386D94033B58C00B384A64013050400E5
:108C9000938504006FF05FE3B7070001130500013F
:108CA000E3E8F6FA130580016FF09FFAB3966601C8
:108CB000335D7601336DDD0033D47901B3956901FD
:108CC00033DC7C0193540D01336CBC0013050400AC
:108CD00093850400B31A6601EF20C032130A050021
:108CE000938504001305040033996C01931C0D0156
:108CF000EF20C02C93DC0C01130405009305050044
:108D000013850C00EF20C028131A0A0113570C0119
:108D10003367EA00130A0400637EA7003307A70144
:108D2000130AF4FF6368A7016376A700130AE4FF40
:108D30003307A701B309A7409385040013850900F1
:108D4000EF20402C938504001304050013850900CF
:108D5000EF20C026930505009304050013850C0041
:108D6000EF20002393150C011314040193D5050182
:108D7000B365B4001387040063FEA500B385A501A5
:108D80001387F4FF63E8A50163F6A5001387E4FFEA
:108D9000B385A501131A0A01B70C0100336AEA0072
:108DA0001384FCFFB3778A0033F48A00B384A540B0
:108DB00013850700930504002326F100135A0A01C6
:108DC000EF20001D930905009305040013050A0018
:108DD000EF20001C13DC0A01930D050093050C0025
:108DE00013050A00EF20C01A8327C100130A0500EB
:108DF00093050C0013850700EF2080193305B5019A
:108E000013D709013307A7006374B701330A9A0126
:108E1000B70701009387F7FF935507013377F700F2
:108E200013170701B3F7F900B3854501B307F7003E
:108E300063E6B400639EB400637CF9003386574157
:108E4000B3B7C700B385A541B385F54093070600C6
:108E5000B307F9403339F900B385B440B3852541F0
:108E600033947501B3D767013365F400B3D5650159
:108E70006FF09FC5370810001308F8FF130101FEBB
:108E8000B378B80013D745019357D50123282101A2
:108E90001379F77F139738003378D800B3E7E700EA
:108EA00013D7460113183800232A91001377F77F50
:108EB00093D8F601232E11009356D601232C81005E
:108EC0002326310193D4F50133E306011315350050
:108ED000131636003308E9406394143B6354001FB3
:108EE000631207143367C3006314070C9306F07F03
:108EF00013070800631CD830B3E6A7006398063058
:108F000093070000130500009396870063DE0600B8
:108F1000130717009306F07F630CD774B70680FF22
:108F20009386F6FFB3F7D7009396D7011355350014
:108F300033E5A6009306F07F93D73700631ED70072
:108F40003365F5009307000063080500B7070800C4
:108F50001305000093040000B70610009386F6FF87
:108F6000B3F7D700B70610801377F77F9386F6FF25
:108F700013174701B3F7D700B3E7E70037070080BF
:108F80001347F7FF8320C101032481019395F40166
:108F9000B3F7E70033E7B700832441010329010158
:108FA0008329C100930507001301010267800000B7
:108FB0009305F8FF639C05043306C5003335A6000E
:108FC000B3876700B387A7001307100013050600D7
:108FD0009396870063DC0622130717009306F07F41
:108FE000E300D7F2B70680FF9386F6FFB3F6D7000B
:108FF00093551500137515009397F60133E5A500F9
:1090000033E5A70093D716006F0040201307F07FC9
:109010006314E80233E7A700630007621307F07FD9
:109020006F00C01E1307F07FE306E9FE37078000DC
:109030003363E3009305080013078003634EB7060C
:109040001307F0016342B704130700023307B74068
:10905000B356B6003318E3003316E6003368D80081
:109060003336C0003368C800B355B3003308A800D6
:10907000B385F500B337A800B387F50013050800E2
:10908000130709006FF0DFF4130700023358B30031
:10909000930600006388E50093060004B385B6409C
:1090A000B316B30033E6C6003336C0003368C800D9
:1090B000930500006FF09FFB3368C3003338000155
:1090C0006FF01FFF630A080E631E0908B3E6A700CE
:1090D000639206029307F07F6318F7003365C300BD
:1090E00093070000E30205E293070300130506005F
:1090F0006F00C0119306F0FF631CD8003305C50054
:10910000B38767003336C500B387C7006FF05FECE5
:109110009306F07F1348F8FFE302D7FC9306800321
:1091200063C606099306F00163CA060593050002AB
:10913000B3850541B3580501B396B7003315B500A3
:10914000B3E616013335A00033E5A60033D8070196
:109150003305C50033086800B337C500B307F8000E
:109160006FF01FE79306F07FE30AD7F6B70680009B
:1091700033080041B3E7D7006FF05FFA93080002AD
:10918000B3D6070193050000630818019305000496
:1091900033880541B395070133E5A5003335A000B9
:1091A00033E5A600130800006FF09FFA33E5A7002F
:1091B0003335A0006FF01FFF130719009375F77F79
:1091C0009306100063C8B60833E7A70063140906C6
:1091D00063080744B366C3001307000063880602F0
:1091E0003306C5003335A600B3876700B387A700F1
:1091F000939687001305060063DA0600370780FFA1
:109200001307F7FFB3F7E700130710009376750015
:10921000E38C06CE9376F50013064000E386C6CEB7
:109220009306450033B5A600B387A7001385060053
:109230006FF09FCD630C073E3368C300E30008DE88
:10924000B7074000130500001307F07F93040000E8
:109250006FF09FCB9306F07FE304D7CA3306C500B7
:1092600033886700B337A6003308F8001315F801F8
:10927000135616003365C500935718006FF01FF999
:10928000635E000F6312070A3367C300E30007C67B
:109290009306F8FF639E06023306C5403335C500CA
:1092A000B3876740B387A740130710001305060074
:1092B00093968700E3DC06F4370480001304F4FF80
:1092C00033F4870093090500130907006F00002796
:1092D0001307F07FE300E8D413078003634AD7083D
:1092E0001307F001634ED704130700023307D7407A
:1092F000B355D6003318E3003316E6003368B800E0
:109300003336C0003368C800B356D3003308054174
:10931000B386D740B3370501B387F640130508007D
:10932000130709006FF0DFF81307F07FE304E9CEBD
:10933000370780003363E300930608006FF0DFF91E
:10934000130700023358D300130400006388E600BB
:1093500013040004B306D4403314D3003366C400AE
:109360003336C0003368C800930600006FF01FFA60
:109370003368C300333800016FF01FFF630A080E23
:10938000631E0908B3E6A700639006029307F07F07
:109390006316F7003365C3006308052A93070300CB
:1093A000130506006F00C00F9306F0FF631ED80080
:1093B0003305A640B307F3403336A600B387C74052
:1093C000938408006FF0DFEE9306F07F1348F8FFF8
:1093D000E302D7FC9306800363C606099306F001F7
:1093E00063CA060593050002B3850541335E050196
:1093F000B396B7003315B500B3E6C6013335A00008
:1094000033E5A60033D807013305A64033080341EE
:10941000B337A600B307F8406FF09FFA9306F07FCA
:10942000E30AD7F6B706800033080041B3E7D70058
:109430006FF05FFA130E0002B3D607019305000028
:109440006308C8019305000433880541B3950701FB
:1094500033E5A5003335A00033E5A600130800006E
:109460006FF09FFA33E5A7003335A0006FF01FFFC0
:10947000130719001377F77F9306100063CAE608F5
:10948000B3E6A7003367C30063140906639E0600B2
:109490006302071C9307030013050600130700006F
:1094A000938408006FF09FD663000704B306C5409D
:1094B000B335D500338767403307B740931587002E
:1094C00063DC05003305A640B307F3403336A6003E
:1094D000B387C7406FF09FFC33E5E600630A050CD5
:1094E0009307070013850600130700006FF01FD2D3
:1094F000639C060063080716930703001305060024
:10950000938408006FF09FB1E30A07B06FF05FD358
:10951000B309C5403384674033383501330404410F
:109520001317840063520708B309A6403304F340BD
:10953000B33736013304F44093840800630E040605
:1095400013050400EF105032130785FF9307F00155
:1095500063CCE70693070002B387E7403314E400C7
:10956000B3D7F90033E487003395E9006340270B54
:1095700033072741930717009306F00163CEF604E3
:10958000130700023307F7403356F500B316E40023
:109590003315E500B3E6C6003335A00033E5A60079
:1095A000B357F4006FF05FF433E58900E31805F872
:1095B000930700006F00800A13850900EF10D02A7E
:1095C000130505026FF05FF8130485FD33948900DD
:1095D000130500006FF09FF9130717FE1306000232
:1095E0003357E400930600006388C7009306000425
:1095F000B386F640B316D4003365D5003335A000EA
:109600003365A700930700006FF01FEEB70780FFD8
:109610009387F7FF3307E940B377F4006FF01FBF7C
:1096200093070300130506006FF01FEC9307030078
:10963000130506006FF09F9E9307000013050000BE
:109640001307F07F6FF05F8C93070000938408008E
:109650006FF09F8B930700001305000013070000B5
:109660006FF0DFBE13050000B70740006FF0DFBDED
:1096700093070000130500006FF01F8B130101FB1F
:1096800023248104232C41033704100013DA4501FD
:1096900023202105232E3103232A51032324810370
:1096A0001304F4FF232611042322910423286103C9
:1096B00023267103232291032320A103232EB1012A
:1096C000137AFA7F13090500130C0600938A06002B
:1096D0003374B40093D9F50163060A0A9307F07F47
:1096E0006304FA1013143400B70780003364F400E5
:1096F000135BD501336B8B0093143500130A1AC02A
:10970000930B000013D54A01370910001309F9FF24
:109710001375F57F3379590193050C0093DAFA013B
:10972000630205109307F07F6302F516370480008B
:1097300013193900336989001354DC01336424019F
:1097400093153C00130515C09307000013972B00D9
:109750003367F7001307F7FF9306E00033C9590199
:10976000330AAA4063E0E61697760100938686B432
:10977000131727003307D700032707003307D70045
:1097800067000700336BA400630E0B06630004043C
:1097900013050400EF10500D930755FF1307C00188
:1097A000634CF702130BD001930485FF330BFB408E
:1097B00033149400335B6901336B8B00B31499004D
:1097C000130AD0C0330AAA406FF09FF3EF10D009FC
:1097D000130505026FF05FFC130485FD331B890040
:1097E000930400006FF0DFFD336BA40063040B02F1
:1097F00093040500130B0400130AF07F930B300051
:109800006FF05FF093040000130A0000930B100048
:109810006FF05FEF93040000130AF07F930B2000BA
:109820006FF05FEE33648901630E04066300090480
:1098300013050900EF105003930755FF1307C001EC
:10984000634EF7021304D001930585FF3304F440FF
:109850003319B90033548C0033642401B315BC00B0
:109860001307D0C03305A7406FF01FEE13050C009F
:10987000EF10807F130505026FF01FFC130485FDB8
:1098800033148C00930500006FF09FFD3364890151
:1098900063020402130409001305F07F93073000EC
:1098A0006FF0DFEA93050000130500009307100036
:1098B0006FF0DFE9930500001305F07F93072000A8
:1098C0006FF0DFE86366640163128B4863E0B448BD
:1098D0009316FB0113D71400139CF401135B1B00B8
:1098E000B3E4E6001314840093DC8501B3EC8C0030
:1098F00093DA0C0193970C0193D70701139D850010
:1099000013050B0093850A002322F100EF10006B72
:1099100093050500930B050013950C0113550501E4
:10992000EF1000671304050093850A0013050B0070
:10993000EF10406D1315050113D704013365A7001F
:1099400093890B00637E8500330595019389FBFFA6
:1099500063689501637685009389EBFF3305950174
:109960003304854093850A0013050400EF10006559
:1099700093050500930B050013950C011355050184
:10998000EF100061130B050093850A001305040016
:10999000EF104067939D04011315050193DD0D0140
:1099A000B3EDAD0013870B0063FE6D01B38D9D0118
:1099B0001387FBFF63E89D0163F66D011387EBFFDF
:1099C000B38D9D0193960901B7040100B3E6E6004B
:1099D000B38D6D41138BF4FF33F76601337B6D015B
:1099E0001305070093050B0013D406012326D100AD
:1099F0002324E100EF10C0592322A10093050B009E
:109A000013050400EF10C058935B0D019309050086
:109A100093850B0013050400EF1080570327810086
:109A20001304050013850B0093050700EF10405643
:109A300003264100330535018326C1001357060173
:109A40003307A7006374370133049400370501001E
:109A50001305F5FF93540701B379A7009399090102
:109A60003376A600B3848400B389C90063E89D00FF
:109A70001384060063949D0463723C05330CAC01AF
:109A80003337AC0133079701B38DED001384F6FF34
:109A900063E6BC016394BC036362AC0363E69D00B0
:109AA000639EB401637C3C01330CAC013337AC01E1
:109AB000330797011384E6FFB38DED00B3093C41F2
:109AC000B3849D40B3373C01B384F4409305F0FF69
:109AD00063889C1A93850A0013850400EF10004EDA
:109AE000930505002324A10013950C0113550501CE
:109AF000EF10004A2322A10093850A001385040079
:109B0000EF10405083268100032741001315050103
:109B100093D7090133E5A700938D0600637EE50026
:109B200033059501938DF6FF636895016376E50033
:109B3000938DE6FF33059501B304E54093850A0054
:109B400013850400EF108047930505002322A10030
:109B500013950C0113550501EF108043130C0500FC
:109B600093850A0013850400EF10C04993990901F9
:109B7000032741001315050193D9090133E5A90015
:109B800093070700637E8501330595019307F7FF6F
:109B900063689501637685019307E7FF33059501B7
:109BA00093940D01B3E4F4009397040193D7070154
:109BB00093050B00B3098541138507002322F100AB
:109BC00093DD0401EF10C03C93050B00930A0500E0
:109BD00013850D00EF10C03B130C050093850D009D
:109BE00013850B00EF10C03A83274100130B0500CB
:109BF00013850B0093850700EF108039330585012D
:109C000093D70A013385A70063768501B707010062
:109C1000330BFB00B70601009386F6FF935705014F
:109C20003377D50013170701B3FADA00B38767015A
:109C30003307570163E8F900938504006390F90442
:109C40006300070433853C019385F4FF6364950347
:109C50006366F5006314F5026370ED0293161D0050
:109C600033BDA601B30C9D019385E4FF3305950137
:109C7000138D06006314F5006304A70193E5150036
:109C80001307FA3F6352E01293F7750063800702EF
:109C900093F7F50093064000638AD700938645004A
:109CA000B3B5B6003304B40093850600931774006F
:109CB00063DA0700B70700FF9387F7FF3374F400F8
:109CC00013070A409307E07F63C2E71A9317D40192
:109CD00093D53500B3E7B70013543400B70610002E
:109CE0009386F6FF3374D400B70610801377F77F9E
:109CF0009386F6FF131747013374D4001319F90143
:109D00003364E400336724018320C1040324810405
:109D100083244104032901048329C103032A810305
:109D2000832A4103032B0103832BC102032C8102ED
:109D3000832C4102032D0102832DC10113850700ED
:109D4000930507001301010567800000130AFAFF5D
:109D5000130C00006FF01FB91389090013040B00E6
:109D60009385040093870B00130720006380E7109E
:109D7000130730006382E70E13071000E392E7F049
:109D800013040000930700006F00400913890A00C4
:109D90006FF09FFD370408009305000013090000D1
:109DA000930730006FF05FFC93061000B386E64027
:109DB00093078003E3C6D7FC9307F00163C4D7067B
:109DC000130AEA41B317440133D7D500339A45014A
:109DD000B3E7E700333A4001B3E747013354D40017
:109DE00013F777006300070213F7F70093064000AC
:109DF000630AD70013874700B337F7003304F40032
:109E00009307070013178400634A07061317D4014A
:109E100093D73700B367F7001354340013070000DB
:109E20006FF0DFEB930710FEB387E74013070002E4
:109E3000B357F400130500006386E600130AEA43F3
:109E400033154401336AB500333A4001B3E74701A3
:109E5000130400006FF0DFF83704080093070000D8
:109E60001307F07F130900006FF05FE71304000091
:109E7000930700001307F07F6FF05FE61304000004
:109E800093070000130710006FF05FE513D745013B
:109E9000B70710009387F7FF13D846019308050012
:109EA000930E05001377F77F1305F07F33F3B700A8
:109EB000130F0600B3F7D70093D5F5011378F87F99
:109EC00093D6F601631AA700336E13011305E0FF62
:109ED000630C0E0867800000631AA80033E6C70011
:109EE0001305E0FF630A0608678000006310070897
:109EF00033651301133515006316080033E6C700F8
:109F000063000606631A0500638ED5001305100072
:109F10006396050067800000E39E06FE1305F0FFD0
:109F200067800000E344E8FE635A07011305F0FF71
:109F3000E38205FE1305100067800000E3E867FC7C
:109F4000631AF300E364DFFD13050000E3E0EEFFB6
:109F50006FF05FFCE36CF3FC13050000678000000A
:109F6000E31C05FE6FF09FFAE30AE8F61305000014
:109F7000E30608F86FF05FF9E31807F8336513019B
:109F8000133515006FF01FF813D74501B707100000
:109F90009387F7FF13D8460193080500930E050039
:109FA0001377F77F1305F07F33F3B700130F060025
:109FB000B3F7D70093D5F5011378F87F93D6F60160
:109FC000631AA700336E130113052000630C0E08FB
:109FD00067800000631AA80033E6C700130520005D
:109FE000630A0608678000006310070833651301E1
:109FF000133515006316080033E6C7006300060634
:10A00000631A0500638ED5001305100063960500E2
:10A0100067800000E39E06FE1305F0FF67800000E6
:10A02000E344E8FE635A07011305F0FFE38205FEEF
:10A030001305100067800000E3E867FC631AF30073
:10A04000E364DFFD13050000E3E0EEFF6FF05FFC6B
:10A05000E36CF3FC1305000067800000E31C05FEC1
:10A060006FF09FFAE30AE8F613050000E30608F82C
:10A070006FF05FF9E31807F8336513011335150026
:10A080006FF01FF8130101FA232C810423263105F8
:10A090003704100093D94501232A91042320610538
:10A0A000232E7103232C81031304F4FF232E1104A8
:10A0B000232821052324410523225105232A910326
:10A0C0002328A1032326B10393F9F97F9304050004
:10A0D000930B0600138C06003374B40013DBF501F8
:10A0E0006388090A9307F07F6386F91037098000B7
:10A0F00013143400336424011359D50133698900E2
:10A10000131D3500938919C0930C000013554C01A1
:10A11000370A1000130AFAFF1375F57F337A8A01A4
:10A1200093840B00135CFC01630405109307F07F1C
:10A130006304F51637048000131A3A00336A8A0064
:10A1400013D4DB013364440193943B00130515C021
:10A150009307000013972C003367F700B389A90019
:10A160001307F7FF9306E000B34B8B01938A1900A6
:10A1700063E0E6169766010093868617131727009B
:10A180003307D700032707003307D700670007000E
:10A190003369A400630E0906630004041305040078
:10A1A000EF00906C930755FF1307C001634CF70253
:10A1B0001309D001130D85FF3309F9403314A401AD
:10A1C00033D9240133698900339DA4019309D0C098
:10A1D000B389A9406FF05FF3EF0010691305050222
:10A1E0006FF05FFC130985FD33992401130D000006
:10A1F0006FF0DFFD3369A40063040902130D05004D
:10A20000130904009309F07F930C30006FF01FF0E6
:10A21000130D000093090000930C10006FF01FEF66
:10A22000130D00009309F07F930C20006FF01FEED8
:10A2300033647A01630E040663000A0413050A00FE
:10A24000EF009062930755FF1307C001634EF702BA
:10A250001304D001930485FF3304F440331A9A00A9
:10A2600033D48B0033644401B3949B009307D0C074
:10A270003385A7406FF0DFED13850B00EF00D05E54
:10A28000130505026FF01FFC130485FD33948B004A
:10A29000930400006FF09FFD33647A0163020402AF
:10A2A00013040A001305F07F930730006FF09FEA54
:10A2B0009304000013050000930710006FF09FE95E
:10A2C000930400001305F07F930720006FF09FE8D0
:10A2D00037070100130AF7FF135C0D0193DD04013A
:10A2E000337D4D01B3F4440193050D001385040043
:10A2F0002328E100EF00D049930C0500938504006A
:10A3000013050C00EF00D0482326A10093850D0013
:10A3100013050C00EF00D047130B050093050D004B
:10A3200013850D00EF00D0468326C10093D70C01A2
:10A330003305D5003385A7006376D50003270101D7
:10A34000330BEB009356050133754501B3FC4C010B
:10A3500013150501B3079501935C0401337444019F
:10A3600093050D0013050400232AD1002326F100D4
:10A37000EF0010422328A1009305040013050C00F0
:10A38000EF001041130A050093850C0013050C0023
:10A39000EF001040130C050093050D0013850C0011
:10A3A000EF00103F032701013305450183264101DA
:10A3B000935707013385A70063764501B70701006E
:10A3C000330CFC003706010093570501338C8701DD
:10A3D0009307F6FF337AF5003377F700131A0A0173
:10A3E000135D0901330AEA003379F9003387460126
:10A3F00093050900138504002328E100232EC100E2
:10A40000EF00103993850400232CA10013050D00E3
:10A41000EF001038232AA10093050D0013850D00CD
:10A42000EF001037930405009305090013850D0014
:10A43000EF00103683264101032781013305D50043
:10A44000935707013385A7006376D5000326C10122
:10A45000B384C400B70601009387F6FF935D05013E
:10A46000B3849D00B37DF5003377F70093050900B1
:10A4700013050400939D0D01B38DED00232CD10035
:10A48000EF00103193050400232AA10013050D00ED
:10A49000EF00103093050D001304050013850C0028
:10A4A000EF00102F130D05009305090013850C0014
:10A4B000EF00102E03274101330585009357070154
:10A4C0003385A7006376850083268101330DDD0087
:10A4D00083270101B70601009386F6FF330BFB00CB
:10A4E000B377D5003377D70093970701B387E70099
:10A4F000333A4B01B387870133844701330BBB01E8
:10A5000033079400B33DBB01B306B70133BC8701E9
:10A5100033344401935705013337970033648C007B
:10A52000B3BDB6013304F400B36DB7013304B40115
:10A530003304A40193D77601131494003364F40018
:10A540008327C10093149B00135B7B01B3E4F400E9
:10A55000B334900093979600B3E46401B3E4F4003D
:10A560009317740063D2071293D7140093F4140066
:10A57000B3E497009317F401B3E4F4001354140008
:10A580001387FA3F6356E01093F774006380070265
:10A5900093F7F40093064000638AD7009387440042
:10A5A000B3B49700330494009384070093177400A6
:10A5B00063DA0700B70700FF9387F7FF3374F400EF
:10A5C00013870A409307E07F63C6E71893DA3400E5
:10A5D0009314D401B3E4540113543400B7071000AA
:10A5E0009387F7FF3374F4009377F77F3707108072
:10A5F0001307F7FF939747013374E400939BFB0124
:10A600003364F400B36774018320C105032481051A
:10A610001385040003290105832441058329C1040E
:10A62000032A8104832A4104032B0104832BC103E1
:10A63000032C8103832C4103032D0103832DC102CD
:10A64000938507001301010667800000930B0B0040
:10A650001304090093040D0093870C0013072000D6
:10A66000638AE70E13073000638CE70C13071000B2
:10A67000E398E7F013040000930400006F008008E3
:10A68000930B0C006FF09FFD938A09006FF05FEF52
:10A6900093061000B386E64093078003E3CCD7FC13
:10A6A0009307F00163C4D706938AEA41B3175401B4
:10A6B00033D7D400B3945401B3E7E700B334900028
:10A6C000B3E497003354D40093F774006380070217
:10A6D00093F7F40013074000638AE7009387440070
:10A6E000B3B4970033049400938407009317840055
:10A6F00063CA07069317D40193D43400B3E49700D8
:10A7000013543400130700006FF05FED930710FE41
:10A71000B387E74013060002B357F40013070000A5
:10A720006386C600938AEA4333175401B3649700E3
:10A73000B3349000B3E49700130400006FF0DFF827
:10A7400037040800930400001307F07F930B000008
:10A750006FF0DFE813040000930400001307F07F9C
:10A760006FF0DFE7130400009304000013071000EC
:10A770006FF0DFE6370810001308F8FF130101FE41
:10A78000B378B80013D745019357D5013378D80073
:10A79000232821011379F77F13973800B3E7E700E7
:10A7A00093D8F60113D74601131838009356D601F3
:10A7B000232A910033E30601232E1100232C81006C
:10A7C000232631011377F77F9306F07F93D4F501A9
:10A7D00013153500131636006316D700B366C30091
:10A7E0006394060093C818003308E9406394983ACC
:10A7F0006354001F631207143367C3006314070C0C
:10A800009306F07F13070800631CD830B3E6A70057
:10A8100063980630930700001305000093968700A5
:10A8200063DE0600130717009306F07F630CD774EE
:10A83000B70680FF9386F6FFB3F7D7009396D7014C
:10A840001355350033E5A6009306F07F93D7370004
:10A85000631ED7003365F500930700006308050009
:10A86000B70708001305000093040000B7061000A6
:10A870009386F6FFB3F7D700B70610801377F77FFC
:10A880009386F6FF13174701B3F7D700B3E7E70046
:10A89000370700801347F7FF8320C101032481019C
:10A8A0009395F401B3F7E70033E7B7008324410140
:10A8B000032901018329C100930507001301010247
:10A8C000678000009305F8FF639C05043306C5000C
:10A8D0003335A600B3876700B387A70013071000BE
:10A8E000130506009396870063DC06221307170002
:10A8F0009306F07FE300D7F2B70680FF9386F6FF5A
:10A90000B3F6D70093551500137515009397F6010C
:10A9100033E5A50033E5A70093D716006F0040206C
:10A920001307F07F6314E80233E7A70063000762B0
:10A930001307F07F6F00C01E1307F07FE306E9FEE8
:10A94000370780003363E300930508001307800393
:10A95000634EB7061307F0016342B7041307000202
:10A960003307B740B356B6003318E3003316E6009A
:10A970003368D8003336C0003368C800B355B3001D
:10A980003308A800B385F500B337A800B387F500F6
:10A9900013050800130709006FF0DFF41307000226
:10A9A0003358B300930600006388E5009306000463
:10A9B000B385B640B316B30033E6C6003336C000E5
:10A9C0003368C800930500006FF09FFB3368C30035
:10A9D000333800016FF01FFF630A080E631E090879
:10A9E000B3E6A700639206029307F07F6318F700AF
:10A9F0003365C30093070000E30205E293070300F9
:10AA0000130506006F00C0119306F0FF631CD80009
:10AA10003305C500B38767003336C500B387C70069
:10AA20006FF05FEC9306F07F1348F8FFE302D7FC6A
:10AA30009306800363C606099306F00163CA060500
:10AA400093050002B3850541B3580501B396B700DD
:10AA50003315B500B3E616013335A00033E5A60083
:10AA600033D807013305C50033086800B337C50084
:10AA7000B307F8006FF01FE79306F07FE30AD7F6FD
:10AA8000B706800033080041B3E7D7006FF05FFAE4
:10AA900093080002B3D6070193050000630818016C
:10AAA0009305000433880541B395070133E5A500FC
:10AAB0003335A00033E5A600130800006FF09FFABD
:10AAC00033E5A7003335A0006FF01FFF130719000F
:10AAD0009375F77F9306100063C8B60833E7A700A5
:10AAE0006314090663080744B366C3001307000034
:10AAF000638806023306C5003335A600B3876700B6
:10AB0000B387A700939687001305060063DA060053
:10AB1000370780FF1307F7FFB3F7E70013071000AD
:10AB200093767500E38C06CE9376F500130640000D
:10AB3000E386C6CE9306450033B5A600B387A700CB
:10AB4000138506006FF09FCD630C073E3368C3008A
:10AB5000E30008DEB7074000130500001307F07F8D
:10AB6000930400006FF09FCB9306F07FE304D7CAF5
:10AB70003306C50033886700B337A6003308F800F2
:10AB80001315F801135616003365C50093571800C6
:10AB90006FF01FF9635E000F6312070A3367C3008B
:10ABA000E30007C69306F8FF639E06023306C5401E
:10ABB0003335C500B3876740B387A740130710003C
:10ABC0001305060093968700E3DC06F43704800043
:10ABD0001304F4FF33F487009309050013090700F9
:10ABE0006F0000271307F07FE300E8D4130780030A
:10ABF000634AD7081307F001634ED7041307000216
:10AC00003307D740B355D6003318E3003316E600B8
:10AC10003368B8003336C0003368C800B356D30079
:10AC200033080541B386D740B3370501B387F640F3
:10AC300013050800130709006FF0DFF81307F07F12
:10AC4000E304E9CE370780003363E300930608008E
:10AC50006FF0DFF9130700023358D300130400002C
:10AC60006388E60013040004B306D4403314D30011
:10AC70003366C4003336C0003368C8009306000052
:10AC80006FF01FFA3368C300333800016FF01FFF05
:10AC9000630A080E631E0908B3E6A7006390060264
:10ACA0009307F07F6316F7003365C3006308052A36
:10ACB00093070300130506006F00C00F9306F0FF13
:10ACC000631ED8003305A640B307F3403336A60011
:10ACD000B387C740938408006FF0DFEE9306F07FE0
:10ACE0001348F8FFE302D7FC9306800363C6060906
:10ACF0009306F00163CA060593050002B38505417A
:10AD0000335E0501B396B7003315B500B3E6C6014F
:10AD10003335A00033E5A60033D807013305A6403C
:10AD200033080341B337A600B307F8406FF09FFA2A
:10AD30009306F07FE30AD7F6B70680003308004198
:10AD4000B3E7D7006FF05FFA130E0002B3D6070126
:10AD5000930500006308C80193050004338805418A
:10AD6000B395070133E5A5003335A00033E5A60010
:10AD7000130800006FF09FFA33E5A7003335A000F9
:10AD80006FF01FFF130719001377F77F930610006A
:10AD900063CAE608B3E6A7003367C3006314090675
:10ADA000639E06006302071C930703001305060059
:10ADB00013070000938408006FF09FD66300070418
:10ADC000B306C540B335D500338767403307B74076
:10ADD0009315870063DC05003305A640B307F340F5
:10ADE0003336A600B387C7406FF09FFC33E5E6001B
:10ADF000630A050C9307070013850600130700007C
:10AE00006FF01FD2639C06006308071693070300C8
:10AE100013050600938408006FF09FB1E30A07B0A2
:10AE20006FF05FD3B309C5403384674033383501D1
:10AE3000330404411317840063520708B309A64082
:10AE40003304F340B33736013304F44093840800ED
:10AE5000630E040613050400EF000021130785FFAD
:10AE60009307F00163CCE70693070002B387E7403E
:10AE70003314E400B3D7F90033E487003395E900D5
:10AE80006340270B33072741930717009306F00110
:10AE900063CEF604130700023307F7403356F5007C
:10AEA000B316E4003315E500B3E6C6003335A00061
:10AEB00033E5A600B357F4006FF05FF433E5890083
:10AEC000E31805F8930700006F00800A1385090056
:10AED000EF008019130505026FF05FF8130485FD7C
:10AEE00033948900130500006FF09FF9130717FED4
:10AEF000130600023357E400930600006388C7007E
:10AF000093060004B386F640B316D4003365D5002B
:10AF10003335A0003365A700930700006FF01FEEE4
:10AF2000B70780FF9387F7FF3307E940B377F40053
:10AF30006FF01FBF93070300130506006FF01FECAF
:10AF400093070300130506006FF09F9E9307000010
:10AF5000130500001307F07F6FF05F8C930700006C
:10AF6000938408006FF09F8B930700001305000087
:10AF7000130700006FF0DFBE13050000B7074000A5
:10AF80006FF0DFBD93070000130500006FF01F8B0B
:10AF9000130605001305000093F6150063840600F0
:10AFA0003305C50093D5150013161600E39605FE6C
:10AFB000678000006340050663C60506138605002A
:10AFC000930505001305F0FF630C060293061000BD
:10AFD000637AB6006358C0001316160093961600E5
:10AFE000E36AB6FE1305000063E6C500B385C540FD
:10AFF0003365D50093D6160013561600E39606FE69
:10B000006780000093820000EFF05FFB138505006E
:10B01000678002003305A04063D80500B305B04047
:10B020006FF0DFF9B305B04093820000EFF01FF935
:10B030003305A040678002009382000063CA0500C8
:10B04000634C0500EFF09FF7138505006780020051
:10B05000B305B040E35805FE3305A040EFF01FF6FE
:10B060003305B04067800200B7070100637AF5023C
:10B070009307F00FB3B7A7009397370013070002A9
:10B080003307F740B357F500175501001305052A9C
:10B09000B307F50003C507003305A740678000002C
:10B0A0003707000193070001E36AE5FC930780017D
:10B0B0006FF0DFFC130101FE232C8100232A910095
:10B0C0001304050093840500232821012326310160
:10B0D0002324410123225101232E1100EF701FB3BD
:10B0E0008327040003290401B7090001B3E5970091
:10B0F000930AC4002320B400930400009389F9FF4D
:10B10000370A00020327040063822A050326090088
:10B1100013050900B3654701B3763601931756004E
:10B1200033F7E6000329490063C6070063160700EA
:10B130006FF05FFDE398E6FC9317760063D4070099
:10B14000B3E4D400EF809FF36FF0DFFB93C4F4FF10
:10B15000B3F4E40023209400EF70DFDE0325040045
:10B160008320C101032481018324410103290101BA
:10B170008329C100032A8100832A410013010102AF
:10B1800067800000130101FF130500002326110052
:10B1900023248100EFC0DFB117C7FFFF1307C7E407
:10B1A00093060000130610009305200317550100B5
:10B1B0001305452CEFA0CFA263020502130405007E
:10B1C000EF705FA61306050013070000930600004A
:10B1D0009305100013050400EFA08FB2EF708FEFFE
:10B1E0008320C10003248100130500001301010125
:04B1F0006780000074
:02000004800278
:10000000FC63FEFF6C65FEFF0864FEFF6C65FEFF8F
:100010006C65FEFF6C65FEFF6C65FEFF3064FEFFE5
:100020006C65FEFF6C65FEFF5864FEFF6864FEFFB2
:100030006C65FEFF8064FEFF9064FEFF9064FEFF2F
:100040009064FEFF9064FEFF9064FEFF9064FEFFEC
:100050009064FEFF9064FEFF9064FEFF6C65FEFFFF
:100060006C65FEFF6C65FEFF6C65FEFF6C65FEFF58
:100070006C65FEFF6C65FEFF6C65FEFF6C65FEFF48
:100080006C65FEFF6C65FEFF6C65FEFF6C65FEFF38
:100090006C65FEFF6C65FEFF6C65FEFF6C65FEFF28
:1000A0006C65FEFF6C65FEFF6C65FEFF6C65FEFF18
:1000B0006C65FEFF6C65FEFF6C65FEFF6C65FEFF08
:1000C0006C65FEFF6C65FEFF6C65FEFF6C65FEFFF8
:1000D0006C65FEFF6C65FEFF6C65FEFF6C65FEFFE8
:1000E0006C65FEFF6C65FEFF6C65FEFF6C65FEFFD8
:1000F0006C65FEFF6C65FEFF6C65FEFF6C65FEFFC8
:10010000D464FEFFFC64FEFF6C65FEFF6C65FEFFC1
:100110006C65FEFF6C65FEFF6C65FEFF6C65FEFFA7
:100120006C65FEFF5C65FEFF6C65FEFF6C65FEFFA7
:100130000C62FEFF1463FEFF6C65FEFF6C65FEFF44
:100140006463FEFF6C65FEFFDC63FEFF6C65FEFF13
:100150006C65FEFF2464FEFFC869FEFF346AFEFF83
:10016000D469FEFF346AFEFF346AFEFF346AFEFF84
:10017000346AFEFF6C68FEFF346AFEFF346AFEFFDD
:100180009468FEFFA468FEFF346AFEFFBC68FEFFB1
:10019000CC68FEFFCC68FEFFCC68FEFFCC68FEFF9B
:1001A000CC68FEFFCC68FEFFCC68FEFFCC68FEFF8B
:1001B000CC68FEFF346AFEFF346AFEFF346AFEFF3D
:1001C000346AFEFF346AFEFF346AFEFF346AFEFFC3
:1001D000346AFEFF346AFEFF346AFEFF346AFEFFB3
:1001E000346AFEFF346AFEFF346AFEFF346AFEFFA3
:1001F000346AFEFF346AFEFF346AFEFF346AFEFF93
:10020000346AFEFF346AFEFF346AFEFF346AFEFF82
:10021000346AFEFF346AFEFF346AFEFF346AFEFF72
:10022000346AFEFF346AFEFF346AFEFF346AFEFF62
:10023000346AFEFF346AFEFF346AFEFF346AFEFF52
:10024000346AFEFF346AFEFF346AFEFF346AFEFF42
:10025000346AFEFF346AFEFF1069FEFF4C69FEFF40
:10026000346AFEFF346AFEFF346AFEFF346AFEFF22
:10027000346AFEFF346AFEFF346AFEFFB869FEFF8F
:10028000346AFEFF346AFEFF4066FEFF9467FEFF9D
:10029000346AFEFF346AFEFF2468FEFF346AFEFF04
:1002A0005068FEFF346AFEFF346AFEFF286AFEFFD4
:1002B000BC9BFEFFD09AFEFFDC9AFEFFD09AFEFFA9
:1002C000A89BFEFFD09AFEFFDC9AFEFFBC9BFEFFC0
:1002D000BC9BFEFFA89BFEFFDC9AFEFFA89AFEFFD8
:1002E000A89AFEFFA89AFEFFE49AFEFF70A3FEFF05
:1002F00070A3FEFF94A3FEFF64A3FEFF64A3FEFFB2
:1003000054A4FEFF94A3FEFF64A3FEFF54A4FEFFCB
:1003100064A3FEFF94A3FEFF60A3FEFF60A3FEFFA5
:1003200060A3FEFF54A4FEFF0001020203030303C7
:100330000404040404040404050505050505050575
:100340000505050505050505060606060606060655
:10035000060606060606060606060606060606063D
:100360000606060606060606070707070707070725
:10037000070707070707070707070707070707070D
:1003800007070707070707070707070707070707FD
:1003900007070707070707070707070707070707ED
:1003A00007070707070707070808080808080808D5
:1003B00008080808080808080808080808080808BD
:1003C00008080808080808080808080808080808AD
:1003D000080808080808080808080808080808089D
:1003E000080808080808080808080808080808088D
:1003F000080808080808080808080808080808087D
:10040000080808080808080808080808080808086C
:10041000080808080808080808080808080808085C
:100420000808080808080808546D72510000000008
:10043000546D722053766300286E756C6C29000031
:100440004572726F7220696E20666C6F70732074D3
:1004500061736B73200D0A006D69616F750A00008E
:100460006D69616F75320A0068756E6772790A008E
:10047000436865636B54696D657200004D61746813
:10048000310000004D617468320000004D617468F5
:0C049000330000004D617468340000006F
:10049C001000000000000000017A5200017C0101F4
:1004AC001B0D020050000000180000008879FEFFB0
:1004BC005805000000440E507489039406990B8172
:1004CC0001880292049305950796089709980A9A51
:1004DC000C9B0D036C010AC144C844C944D244D3DB
:1004EC0044D444D544D644D744D844D944DA44DB24
:1004FC00440E00440B0000004C0000006C00000097
:10050C008C7EFEFFDC05000000440E3070890395E4
:10051C00078101880292049305940696089709981E
:10052C000A990B9A0C0370020AC144C844C944D2FC
:10053C0044D344D444D544D644D744D844D944DADB
:10054C00440E00440B00000050000000BC000000F2
:10055C001884FEFF0005000000440E5074880289C8
:10056C00039305990B8101920494069507960897BD
:10057C0009980A9A0C9B0D0320010AC144C844C96E
:10058C0044D244D344D444D544D644D744D844D993
:0C059C0044DA44DB440E00440B00000075
:100618006AE67F50274C41C15305A3923ADD5E40FC
:1006280082E2C7985B53A240B29DEFA7C6B18CC0C7
:10063800FCA9F1D24D62503FAE47E17A145678C01A
:10064800CDCCCCCC8CBCDF4039D6C56D340000C0D5
:10065800E5D022DBF93E2840E5D022DBF93E3840E0
:10066800AC1C5A643B2F4240E5D022DBF93E48409F
:100678001E85EB51B84E4E40AC1C5A643B2F52407D
:10068800C876BE9F1A375540E5D022DBF93E584060
:10069800022B8716D9465B40FCA9F1D24D6250BFA8
:1006A80000000000000016400000000000001A4092
:1006B8000000000000001E40000000000000214073
:1006C800000000000000234000000000000025405A
:1006D8000000000000002740000000000000294042
:1006E8000000000000002B400000000000002D402A
:0806F800FC8F0100040000006A
:040000058000004037
:00000001FF
